:020000040000FA
:06080000D3EF39F01200F5
:06080800E1EF26F01200F2
:06082A00060053740000FB
:1008300090030000040000003174000096020000E4
:1008400022000000097400006E0200002800000071
:1008500007740000FE00000002000000F0730000BA
:100860001703000017000000E073000044030000BD
:040870001000000074
:0C0874000901006B0A0E005D26E2005135
:10088000220DF3CF01F9F4CF02F9000E01270A0E71
:100890000223DFEC0CF0EF6A34EC0EF0EF9034EC56
:1008A0000EF0EF8234EC0EF0EF8434EC0EF0EF98A3
:1008B00034EC0EF0EF96DFEC0CF0EFEC0DF0DFEC2B
:1008C0000CF003EC0EF0002BD7D70101496B040E9E
:1008D0004A6F4B6B4C6B4D6B4E6B12000901006BFA
:1008E0000A0E005D36E20051220DF3CF01F9F4CF7C
:1008F00002F9000E01270A0E0223CEEC0CF0EF5095
:10090000000925E1CEEC0CF0010EEF6ECEEC0CF000
:100910000B0E4FC1EBFF0C0E50C1EBFFCEEC0CF0F9
:100920000D0EEB6A0E0EEB6ACEEC0CF0FFEC0DF048
:1009300046EC0EF0EF8046EC0EF0EF96CEEC0CF0AD
:10094000EFEC0DF046EC0EF0EF8200511200002BA0
:10095000C7D7FE0C09016F6B6C6B0A0E6C5D14E25D
:100960006C51220DF3CF6DF9F4CF6EF9000E6D27A7
:100970000A0E6E2385EC0CF0EF50000903E1010E26
:100980006F6F02D06C2BE9D76F5101E1FE0C0101B2
:10099000492B000E4A2385EC0CF00B0E49C1EBFFEE
:1009A0000C0E4AC1EBFF880ED8804955130E4A55EC
:1009B00003E2496B040E4A6F85EC0CF0A1EC0DF0DC
:1009C000EF9085EC0CF00D0E53C1EBFF0E0E54C1F1
:1009D000EBFF4B2B000E4C234D234E2307EC0EF068
:1009E00043EC0DF085EC0CF0180E6DEC0CF067ECA0
:1009F0000DF00A0EE66EE66A51C1E6FF52C1E6FF4F
:100A000085EC0CF08FEC0CF0F9EC0CF00101020E0F
:100A10007E6F85EC0CF0F3EC0DF007EC0EF0E9ECDA
:100A20000CF085EC0CF0F7EC0DF085EC0CF0FBEC29
:100A30000DF085EC0CF0D8EC0CF085EC0CF0030E0E
:100A4000EF6E07EC0EF093EC0DF085EC0CF0F2EC91
:100A50000CF009016C51120001015551A8EC0CF089
:100A6000EF50040801E0000C010C01015651220D69
:100A7000F3CF81F9F4CF82F9000E090181270A0E24
:100A80008223E4EC0CF0EF50040806E081C988F101
:100A900082C989F1CCEF0AF056C160F14CD9F9EC6A
:100AA0000CF00101110E7E6FE4EC0CF0F3EC0DF094
:100AB000E4EC0CF037EC0EF0E9EC0CF0E4EC0CF0AC
:100AC000F7EC0DF0E4EC0CF0FBEC0DF0E4EC0CF0CA
:100AD000D8EC0CF0E4EC0CF037EC0EF093EC0DF0ED
:100AE000E4EC0CF0050EEF6E120001015751220DDF
:100AF000F3CF83F9F4CF84F9000E090183270A0E9E
:100B000084238AEC0CF09DEC0DF001E1000C8AECE2
:100B10000CF023EC0EF0020B01E1000C8AEC0CF05F
:100B2000100E6DEC0CF0EECF80F1EDCF81F18AEC80
:100B30000CF00F0EEB5001017F6F0101100E7E6F64
:100B4000F3EC0DF08AEC0CF037EC0EF0E9EC0CF065
:100B50008AEC0CF0F7EC0DF08AEC0CF0FBEC0DF0ED
:100B60008AEC0CF0D8EC0CF08AEC0CF0100EC8EC0F
:100B70000DF0126A136A8AEC0CF037EC0EF010508C
:100B8000EE261150EE221250EE221350EE2255ECBA
:100B90000EF0EF9255EC0EF0EF988AEC0CF022EC90
:100BA0000DF08AEC0CF0EFEC0DF055EC0EF0EF824E
:100BB000010C0A0E0101585D13E25851A8EC0CF02B
:100BC0000F0E6DEC0CF0EF50FF0802E166EF18F02D
:100BD0005851A8EC0CF023EC0EF0020B02E0010CD3
:100BE000000E120001015951220DF3CF81F9F4CF0B
:100BF00082F9000E090181270A0E8223D3EC0CF042
:100C00009DEC0DF014E1D3EC0CF00F0E1BC0EBFFCC
:100C1000D3EC0CF0EB500201596F9EEC19F0D3ECC1
:100C20000CF04CEC0DF0D3EC0CF07BEC0DF0D3ECB5
:100C30000CF026EC0EF001E3000CD3EC0CF0A1EC70
:100C40000DF0EF885AC150F274EC18F0D3EC0CF0B0
:100C5000100E6DEC0CF0EE2AEF22D3EC0CF026EC2B
:100C60000EF003E359C157F140DF010C01015B5164
:100C7000220DF3CF6CF9F4CF6DF9000E09016C274A
:100C80000A0E6D23B7EC0CF09DEC0DF014E1B7ECFF
:100C90000CF00F0E1BC0EBFFB7EC0CF0EB50020199
:100CA000596F9EEC19F0B7EC0CF04CEC0DF0B7EC72
:100CB0000CF07BEC0DF0B7EC0CF026EC0EF001E341
:100CC000000C0DEC0EF0EE24106E5F51EE20116E54
:100CD000CA0ED8801054030E11540EE2B7EC0CF07B
:100CE000100E6DEC0CF0EECF5EF1EFCF5FF1CA0E9F
:100CF000D8805E57030E5F57B7EC0CF0A1EC0DF0F7
:100D0000EF885EC153F25FC154F25CC151F25DC124
:100D100052F296EC18F00DEC0EF0EE265F51ED223B
:100D2000B7EC0CF026EC0EF003E35BC157F1DDDE0F
:100D300001015E51120001016051220DF3CF00F953
:100D4000F4CF01F9000E090100270A0E012300C9A2
:100D5000E9FF01C9EAFF52EC0EF001E1000CACEC36
:100D600019F000C9E9FF01C9EAFFA1EC0DF0EF9607
:100D7000010C01016151220DF3CF20F9F4CF21F9CB
:100D8000000E090120270A0E212318EC0DF052EC69
:100D90000EF02BE018EC0DF023EC0EF0040B08E045
:100DA000280E1DEC0DF018EC0DF0A1EC0DF0EF94F9
:100DB00018EC0DF04CEC0EF0EE50ED1008E1ACEC40
:100DC00019F018EC0DF0A1EC0DF0EF96000C18ECFA
:100DD0000DF04CEC0EF0EE06EF5A14EC19F062C177
:100DE000E9FF63C1EAFFEF6E010C000C01016451E1
:100DF000220DF3CF02F9F4CF03F9000E0901022707
:100E00000A0E0323FFEC0CF052EC0EF03AE0FFEC7C
:100E10000CF023EC0EF0040B08E0280E1DEC0DF096
:100E2000FFEC0CF0A1EC0DF0EF94FFEC0CF0120EC7
:100E3000C8EC0DF001016751105C6851115808E2CF
:100E4000FFEC0CF04CEC0EF0EECF67F1EDCF68F15B
:100E5000FFEC0CF04CEC0EF0EE50ED1008E1ACECB9
:100E600019F0FFEC0CF0A1EC0DF0EF960AD067C181
:100E700057F268C158F265C155F266C156F252EF99
:100E800019F0F36AF46A12000A0E0101695D07E2C3
:100E90006951A8EC0CF052EC0EF002E0010C000ECF
:100EA00012000901736B6C6B0A0E6C5D01E3D4D008
:100EB0006C51220DF3CF6DF9F4CF6EF9000E6D2752
:100EC0000A0E6E237BEC0CF052EC0EF001E0C1D068
:100ED0007BEC0CF023EC0EF0100B01E0BAD07BECB5
:100EE0000CF0EF50000901E1B4D07BEC0CF0EF50B6
:100EF000010807E17BEC0CF023EC0EF0010B01E0A4
:100F0000A8D07BEC0CF01D0E6DEC0CF00301EE5044
:100F1000855D106EEE508659116E7BEC0CF01F0E45
:100F20006DEC0CF071EC0DF01050125C1150135878
:100F300001E38FD066EC18F0000901E112007BECB0
:100F40000CF0F2EC0CF07BEC0CF01F0E6DEC0CF0E6
:100F5000EE2AEF227BEC0CF01C0E6DEC0CF0EF2A6D
:100F60007BEC0CF0EF50060A27E0010A25E0020AAC
:100F70001CE00F0A1AE00E0A10E0060A05E0010A5A
:100F800028E10901020E24D013EC0EF0106E030EBE
:100F9000105C16E20901120E1BD00901110E736FCD
:100FA0007BEC0CF0050EEF6E14D013EC0EF0030882
:100FB00007E30901010E0CD013EC0EF0030806E262
:100FC0006DC988F16EC989F1E7DA03D00901100E05
:100FD000736F0901735100083CE2100E735D11E05C
:100FE0007BEC0CF037EC0EF0EFCF6FF9EE2AEFCF81
:100FF00070F9EE22EFCF71F9EE22EFCF72F9EF2206
:101000000CD07BEC0CF037EC0EF0EECF6FF9EECF9E
:1010100070F9EECF71F9EFCF72F9F9EC0CF073C9FA
:101020007EF17BEC0CF0F3EC0DF06FC976F170C93A
:1010300077F171C978F172C979F17BEC0CF0F7ECBA
:101040000DF07BEC0CF0FBEC0DF07BEC0CF0D8EC35
:101050000CF009016C2B28D71200140E0201576FF7
:10106000586B02016C0E556F090E566F52EC19F059
:1010700001016C0E866F090E876F59DA6AC1E9FFAC
:101080006BC1EAFF4FEC0EF0EECF80F9EECF81F9A5
:10109000EECF82F9EFCF83F998EC0DF0EFCF84F922
:1010A000010E6DEC0CF0EFCF85F998EC0DF0020E0F
:1010B0006DEC0CF0EFCF86F998EC0DF0030E6DECB3
:1010C0000CF0EFCF87F90901886B060E896F6EC1AE
:1010D0008AF96FC18BF96EC1D8F26FC1D9F27EEC7B
:1010E0002AF0F3CF8AF9F4CF8BF90C0E0201E06FEE
:1010F000E16B0201800EDE6F090EDF6FB2EC2AF0A9
:10110000F3CF8DF9F4CF8EF909018D1F8E1F240EB8
:101110001DEC0DF08DC950F274EC18F08EC950F230
:1011200074EC18F0140E1DEC0DF06EC1E2F26FC1FC
:10113000E3F20EEC2BF0F3CF8DF9F4CF8EF9090129
:101140007C51F31802E17D518E1903E0ACEC19F0EB
:10115000010C55EC0DF0106E116A140E105E000EAD
:10116000115A10C08FF91050106E116AE850010129
:101170006E5D6E6F11506F596F6F140E6E5F000EC3
:101180006F5B090155EC0DF00201696F6A6B140E7B
:101190006927000E6A2349EC1BF06AC184F16BC118
:1011A00085F101016C0E826F090E836F3ED9090132
:1011B0008C6FFE0E8C5D11E26EC18FF16FC190F1EC
:1011C00001016C0E8D6F090E8E6F6AC18BF16BC1C0
:1011D0008CF18CC98AF106DA010CACEC19F0FF0E27
:1011E00009018C5D37E101016E510901742701018C
:1011F0006F5109017523000E762377237951020B75
:1012000003E17951010B05E0742B000E7523762361
:101210007723EFDB0101040E7E6F70C97AF171C98B
:101220007BF172C97CF173C97DF174C976F175C91E
:1012300077F176C978F177C979F16CC974F16DC924
:1012400075F16EC972F16FC973F16AC170F16BC14A
:1012500071F101D8010C72C148F973C149F974C127
:101260004AF975C14BF976C14CF977C14DF978C18E
:101270004EF979C14FF97AC150F97BC151F97CC15E
:1012800052F97DC153F909015491549354955497DF
:101290007EC155F9BFEC19F0F3CF56F9F4CF57F9E9
:1012A0000901000EF35C040EF45804E3566B040EBF
:1012B000576F0DD0360ED8805655000E575505E2A3
:1012C000360E565F000E575B02D0566B576B586B4D
:1012D000596B5A6B5B6B0101480E866F090E876F65
:1012E00026D9140E01018027000E81237EA30ED083
:1012F000040E8027000E81230901020E5C6F040E8C
:101300005D6F5E6F5F6B5499548B03D009015489F4
:10131000549B548D549FB8C260F9B9C261F9BAC2E6
:1013200062F9BBC263F970C1E9FF71C1EAFF4FEC1A
:101330000EF0EECF64F9EECF65F9EECF66F9EFCFA0
:1013400067F9686B060E696F80C16AF981C16BF934
:1013500080C1D8F281C1D9F27EEC2AF0F3CF6AF9CC
:10136000F4CF6BF90C0E0201E06FE16B0201600E2D
:10137000DE6F090EDF6FB2EC2AF0F3CF58F9F4CF2D
:1013800059F90901581F591F58C946F959C947F950
:10139000FF0E01017F5D02E11BC07FF1140E41DBF6
:1013A00080C16EF381C16FF30301060E6D6F70C1D2
:1013B0006BF371C16CF3E9EC2CF0140E0201536F66
:1013C000546B0201480E516F090E526F96EC18F0E3
:1013D00001017EA30BD0040E0201536F546B020176
:1013E0005C0E516F090E526F96EC18F0140E19DB5B
:1013F00080C1E2F281C1E3F20EEC2BF0F3CF46F9AB
:10140000F4CF47F9240E0DDB47C950F274EC18F005
:1014100046C950F274EC18F002016C6B6D6B7FC121
:101420006BF25CEC1BF0FBEF1AF00901FE0E036F90
:10143000026B0A0E025D4AE202511BDB84DAEF50B6
:10144000000941E080DA0B0EA3DB50DB020E45DA27
:1014500048DB00011250101836E11350111833E127
:1014600072DAEF50010802E102C903F96CDA0D0EDD
:101470008FDB3CDB36DB1250101825E113501118BE
:1014800022E184C1E9FF85C1EAFF4FEC0EF0EECF07
:1014900014F0EECF15F0EECF16F0EFCF17F053DAD1
:1014A000EE524FEC0EF0EE5014180DE1EE50151800
:1014B0000AE1EE50161807E1EE50171804E103E1B7
:1014C0000901025112000901022BB3D70351D1DAED
:1014D000FE0E035D27E037DAEF50010823E10A0E24
:1014E000E66EE66A84C1E6FF85C1E6FF2CDA17DA0C
:1014F0001250FCDA020E4CDB26DA0B0E10C0EBFFAA
:101500000C0E11C0EBFFF2DA2DDA1DDAFADA1BDA73
:1015100018DBEF9618DA63DB16DA13DBEF820901CA
:1015200003511200FE0E035D01E1FF0CFE0CDED93B
:10153000EFCF07F9A2DBE552E750EF6ED7D92BDBEF
:10154000020E35DB020E09DB020E2BDB020EA1DBE5
:10155000040E09DB040E30DB080E05DB080E2CDB65
:101560000E0E25DB0E0EF9DA0E0E1BDB0E0E91DBD6
:10157000100E1DDB100EF1DA100E13DB100E89DBDE
:10158000120E15DB120EE9DA120E0BDB85DB010EF3
:10159000A4D907C9EFFF1200D1D9CFDA06E0CED91E
:1015A00051DACCD91CDB84DBEF82C8D928DBC6D961
:1015B0000D0EEB6A0E0EEB6AC1D974DB02E0ACECE7
:1015C00019F076DBEF96BAD91EDB72DBEF98B6D94D
:1015D0003ADB010B04E0B2D9010EEF6E1200AED976
:1015E000EF6A12000901A26B01018A51220DF3CFAB
:1015F000A0F9F4CFA1F9000E0901A0270A0EA1233A
:10160000A8DAEECF98F9EECF99F9EECF9AF9EFCFAD
:101610009BF9A6DAEECF9CF9EECF9DF9EECF9EF9BD
:10162000EFCF9FF96DD9040E58D948DA01018F51D7
:10163000090190270101905109019123000E922385
:10164000932308DBC4DADFDAE5DA01083AE1ACEC2F
:1016500019F001014B2B000E4C234D234E2380DA51
:1016600012DA0901902B91239223932303DBF2DA00
:1016700077DA59DA69DA020B14E00A0EE66EE66AE6
:101680008BC1E6FF8CC1E6FF2CD949D9125038D95D
:1016900069D927D936DA0901120EA26F22D9020EB2
:1016A000DCD0040EA26F90C994F991C995F992C942
:1016B00096F993C997F924D910D900DA12D99FDA8B
:1016C000D9D042DA040B04E0ACEC19F088EF0DF04D
:1016D00017D9080E02D99451EE1801E0C9D09551DE
:1016E000EE1801E0C5D09651EE1801E0C1D0975137
:1016F000EE1801E0BDD001E0BBD08CDA02080AE1AF
:10170000C2DA01E1B5D0B6DA62DA040EEF6EA0D922
:101710002CE3AED07FDA03082AE116DA020B01E1EE
:10172000A7D0902B000E912392239323A3DAABDA58
:1017300006E0100EA26FD5D8040EEF6E13D0120E75
:10174000A26FCFD8020EEF6E942B000E9523962336
:10175000972306DA94C9EEFF95C9EEFF96C9EEFF0E
:1017600097C9EEFF75D901E383D061DA83D0C8D879
:10177000040EB3D8EECF10F0EECF11F0B2D9E9D904
:101780001050EE1808E11150EE1805E11250EE1855
:1017900002E11350EE1802E0ACEF19F06BDA3ADA1E
:1017A000040842E170DA09E09CD8C7D906E099D86C
:1017B00049D997D814DA7FDAEF82C6D9010B15E040
:1017C0000901110EA26FCCD9EFCF94F9EE2AEFCF19
:1017D00095F9EE22EFCF96F9EE22EFCF97F9EF22AF
:1017E000B8D912D97ED80A0EEF6E32D941E279D833
:1017F00059DA05E11CDA0901100EA26F3BD009018C
:10180000A26BAED99CC9EEFF9DC9EEFF9EC9EEFF4B
:101810009FC9EEFF9ED998C9EEFF99C9EEFF9AC9FC
:10182000EEFF9BC9EEFF24D0F5D90A0805E1ACEC28
:1018300019F029DA1FE01AD0EDD9050810E1ACEC57
:1018400019F082D9010B16E00901100EA26F81D99F
:10185000DBD819DA0BE145D8060EEF6E0BD0DAD9DA
:10186000060808E1ACEC19F00EDA04E051D902D018
:10187000ACEC19F00901A25100081EE2BAD8A2C9C5
:101880007EF190C97AF191C97BF192C97CF193C93B
:101890007DF194C976F195C977F196C978F197C928
:1018A00079F12ED8DCD82CD8020E17D8DDD88BC110
:1018B00070F18CC171F1CFDC120001019151220D48
:1018C000F3CF10F0F4CF11F0000E10260A0E112203
:1018D00010C0F3FF11C0F4FF1200E926000EEA2247
:1018E0001200A0C9E9FFA1C9EAFF120086C1E9FF01
:1018F00087C1EAFF12006DC9E9FF6EC9EAFF120055
:101900008DC1E9FF8EC1EAFF12006DC9E9FF6EC902
:10191000EAFF120083C9E9FF84C9EAFF1200EE5210
:10192000E9CF10F0EACF11F0E9CFE6FFEACFE6FF0A
:10193000AAEC35F0126E060EE15E120088C1E9FFD6
:1019400089C1EAFF120000C9E9FF01C9EAFF1200DC
:10195000220DF3CFE9FFF4CFEAFF000EE9260A0ECD
:10196000EA221200EECF10F0EFCF11F012006CC996
:10197000E9FF6DC9EAFF1200EECF7AF1EECF7BF1FD
:10198000EECF7CF1EFCF7DF1120090C9EEFF91C94F
:10199000EEFF92C9EEFF93C9EEFF120001C9E9FF05
:1019A00002C9EAFF120081C9E9FF82C9EAFF1200F9
:1019B000EE52E9CF70F1EACF71F12BEF09F001C9D6
:1019C000E9FF02C9EAFF120081C9E9FF82C9EAFF03
:1019D0001200EECF76F1EECF77F1EECF78F1EFCFC8
:1019E00079F112001D0E85C3EBFF1E0E86C3EBFFBF
:1019F00012000101806B816B01017F69120002C935
:101A0000E9FF03C9EAFF1200EF2AEECF90F9EF22B7
:101A1000EECF91F9EF22EECF92F9EF22EFCF93F9CB
:101A2000120002016C6F6D6B7FC16BF25CEF1BF0FB
:101A300020C9E9FF21C9EAFF12000201696F6A6B40
:101A400049EF1BF00F0EEB5002015A6FA4EF19F093
:101A50000101000ED8808F55000E90551200EECF78
:101A600074F1EDCF75F11200EECF72F1EDCF73F19D
:101A70001200220DF3CF00F9F4CF01F9000E002778
:101A80000A0E012312004BC1EEFF4CC1EEFF4DC107
:101A9000EEFF4EC1EEFF1200100EEB6A110EEB6A64
:101AA000280E02016C6F6D6B12007851F00BE8424A
:101AB000E842E842E842040DF3501200EECF90F9FC
:101AC000EECF91F9EECF92F9EFCF93F91200EE6AD3
:101AD000EE6AEE6AEE6A1200CA0E105C030E11582E
:101AE0001200EECF12F0EFCF13F0120082C1E9FF27
:101AF00083C1EAFF12000F0EEB5002016B6F5CEF27
:101B00001BF00D0E10C0EBFF0E0E11C0EBFF12000C
:101B1000A0C988F1A1C989F1CCEF0AF0700EEE6E70
:101B2000170EED6E1200EE2AEE22EE22EE221200C9
:101B30006CC1E9FF6DC1EAFF12000F0EEB50FF0808
:101B40001200210E6DEF0CF0DBDE0D0EC6DEEF5045
:101B50001200C7DE180E6DEF0CF0BFDE3DEF0EF089
:101B6000C0DE37EF0EF0B9DEEECFDAF2EECFDBF209
:101B7000EECFDCF2EFCFDDF283EC2AF004C010F000
:101B800005C011F006C012F007C013F076EF0CF09C
:101B9000A4DEB2EF0CF0010EA0DE07C9EFFF76EF76
:101BA0000CF09BDEE552E750EF6E76EF0CF095DE21
:101BB000EFCF07F976EF0CF090DE04C0EEFF11C016
:101BC000EEFF12C0EEFF13C0EEFF76EF0CF089DEE1
:101BD0001C0E83DEEF6A85DE05DF71EF0CF00F0E61
:101BE0007CDEEF681200180E78DEBCEF0CF00D0EF4
:101BF00074DE2FEF0DF00B0E70DE34EF0DF0EE52B1
:101C00004ED867EF0DF01F0E68DE8EEF0DF07DDE13
:101C100037EF0EF066DEEF501200A9DE100E5DDE2B
:101C200001015E51120067DE1C0EEB50120043D81A
:101C3000EF8657DE120E8FC1EBFF130E90C1EBFF44
:101C40003AD8EF8412007DDFEF501200100EA0DFB3
:101C50006CEF0DF085DFEECF94F9EECF95F9EECF76
:101C600096F9EFCF97F91200AADEA1EF0DF0140E4E
:101C70006DEF0CF06EDFC5EF0CF0010E2EDEEF50B5
:101C8000E66E76EF0CF060DF100B120087DEA1EF3E
:101C90000DF023DECBEF0DF0120E6DEF0CF0060E03
:101CA0006DEF0CF0D0DF080B120034DEA1EF0DF069
:0C1CB00045DEA1EF0DF015DEA1EF0DF0F8
:041CBC001200F0EC36
:101CC00012F0040B06E0F0EC12F0080B01E0020C3D
:101CD000010C000C09011C6B1D6BE2C1E9FFE3C1A3
:101CE000EAFFEF506B0801E080D00901010E206F80
:101CF0000201210EE76F090EE86F010E0101E225D6
:101D00000201E56F000E0101E3210201E66F88EC9C
:101D10002BF0000903E1F36AF46AB1D1E4C1E6FFF4
:101D2000E5C1E6FF69EC31F0E552E552F3CF22F967
:101D300009012151110804E2160E0901215D05E196
:101D400009011C830901206B43D0090121511508A9
:101D500009E3130E0901215D04E009011C8F09014B
:101D6000206B36D0090121511A0801E331D0090155
:101D700021511E0801E32CD009012151220817E34B
:101D80001F0E0901215D04E0210E0901215D07E11B
:101D900009012251080802E30901206B02D0090160
:101DA000206B0901205102E109011C8511D00901B4
:101DB0002151300805E309011C870901206B08D077
:101DC00009012151320804E309011C890901206B32
:101DD0000901205109E10101E65106E022C9A8FFED
:101DE00021C9D7F2A0EC36F045D1E2C1E9FFE3C149
:101DF000EAFFEFCF10F0610E105C01E2B5D0E2C156
:101E0000E9FFE3C1EAFFEF50670801E2ADD0E2C1AC
:101E1000E9FFE3C1EAFFEF50640807E0E2C1E9FF30
:101E2000E3C1EAFFEF50650803E1F36AF46A27D1E2
:101E3000E2C1E9FFE3C1EAFFEF509F0F09011E6F06
:101E40001F6B890E09011E270F0E09011F23010EAA
:101E50000101EA6AE225E96EE351EA22EF5014E15A
:101E60000201200EE76F090EE86FE4C1E5F2E5C15B
:101E7000E6F288EC2BF0000906E01EC9E9FF1FC955
:101E8000EAFF20C9EFFF6FD0010E0101EA6AE225E7
:101E9000E96EE351EA22EF50780833E1020E0101C6
:101EA000EA6AE225E96EE351EA22EF50D00F106EA4
:101EB000010E105204E0E846FE0B1006FCE1090199
:101EC000206FE4C1E9FFE5C1EAFFEF5031080AE104
:101ED0000901201D106E1EC9E9FF1FC9EAFF10503D
:101EE000EF160ED0E4C1E9FFE5C1EAFFEF5030087C
:101EF00007E11EC9E9FF1FC9EAFF09012051EF12DE
:101F000032D0010E0101EA6AE225E96EE351EA22CC
:101F1000EF50D00F106E010E105204E0E846FE0B99
:101F20001006FCE10901206FE4C1E9FFE5C1EAFF09
:101F3000EF5030080AE10901201D106E1EC9E9FFAB
:101F40001FC9EAFF1050EF160ED0E4C1E9FFE5C14A
:101F5000EAFFEF50310807E11EC9E9FF1FC9EAFF98
:101F600009012051EF1286D0E2C1E9FFE3C1EAFF87
:101F7000EF506C082DE10101E65129E0010E01014D
:101F8000EA6AE225E96EE351EA22EF50610A11E0C4
:101F9000030A01E01CD00201080EED6FE4C1EBF270
:101FA000E5C1ECF23E0E0201E96FEA6BADEC2BF0FD
:101FB0000ED00201080EED6FE4C1EBF2E5C1ECF2C8
:101FC000350E0201E96FEA6BADEC2BF000D052D078
:101FD000E2C1E9FFE3C1EAFFEF506D081AE1010138
:101FE000E65116E0E4C1E9FFE5C1EAFFEF50720AED
:101FF00001E00ED005EC1BF0FF0E986E966E956E0C
:10200000936E000E866E846E836E816EFF0000D02C
:1020100031D0E2C1E9FFE3C1EAFFEF507A082AE1DB
:102020000201230EE76F090EE86F010E0101E225A0
:102030000201E56F000E0101E3210201E66F88EC69
:102040002BF0000903E1F36AF46A19D0E4C1E6FF5A
:10205000E5C1E6FF69EC31F0E552E552F3CF24F932
:10206000F4CF25F924C9F9F225C9FAF223C9F8F207
:1020700066EC27F01CC9F3FF1DC9F4FF00D0120065
:102080000901146B156B186BE7C1E0F1E8C1E1F1D0
:1020900016DE0901196F140E166F0B01160EB46FC0
:1020A000090EB56F0B01000EB26F090EB36FB1DAF6
:1020B000EF500B01B16F5EEC15F00901176F182B93
:1020C0001B6B6C0E005D36E10151750A2BE0050AB1
:1020D00045E1010E1B6F3E0E54DA40E1020E09018C
:1020E000185D3CE1010E1A1539E093DAEF50010159
:1020F000916F5DEC0CF0F3CFE9FFF4CFEAFFEE5205
:10210000060E83DAEECFA6FBEECFA7FBEECFA8FB41
:10211000EFCFA9FB0B01010EAA6F43DAEF8441DA7E
:10212000EF961CD0010E1B6F350E2BDA17E109015B
:102130001A8114D06D0E005D11E119510FE0165196
:10214000EA6A000FE96E090EEA22EF506F0A06E113
:10215000010E1B6F0B01AA6B24DAEF9409011B51CE
:1021600015E119C9E6F116510101E46FE56B000EA6
:10217000E427090EE5230101000EE26F090EE36F6B
:10218000A9DDF35009011413F4501513175101E0A0
:1021900082D71451020B01E012001451040B02E02B
:1021A000B4EF36F01451080B02E003EF37F014518E
:1021B000100B02E02FEC37F01200F7D9020E25DAEF
:1021C000EFCF01F9F2D9030E20DAEFCF02F9EDD902
:1021D000EECF07F9EDCF08F913DAEF6AEBC1E0F1C2
:1021E000ECC1E1F16CDD0901096F610E025D6DE387
:1021F000025168086AE3006B610E025D066F070E0C
:102200000115106E010E105204E0E846FE0B100698
:10221000FCE10901056F0651036F046B920E032761
:102220000F0E0423D0D909E10651036F046B890E08
:1022300003270F0E0423008107D00651036F046BA0
:10224000800E03270F0E0423F00E0115066FE850D1
:1022500004E1B9D934E0310E35D0100E065D0CE141
:10226000B2D905E10101CC0EF26F720E02D101016B
:10227000C90EF26F720EFDD0200E065D03E1010E55
:10228000001506E0300E065D08E1010E001505E0C0
:10229000080E011501E1D8D0E8D0400E065D08E136
:1022A000010E001505E00101AF0EF26F720EE1D0D4
:1022B000500E065D01E0E6D0010E001502E0300E82
:1022C00001D0310E9DD9EF6EDDD06B0E025D0AE1BB
:1022D000095101E1D7D001C9D6F296EC36F00101DF
:1022E000FC6F62D06C0E025D42E109512CE001519D
:1022F000040A24E0060A1DE0030A16E0010A01E0D0
:10230000C1D009050CE1350E0101F76FF86BEDC185
:10231000F5F1EEC1F6F107C9F4F164EF12F0010135
:102320003A0EF26F5C0EA5D00101D40EF26F730E5F
:10233000A0D00101DA0EF26F730E9BD00101360EB0
:10234000F26F5C0E96D00151030A08E0030A01E027
:1023500099D00101300EF26F5C0E8BD0095102E171
:10236000300E01D0310E066FE8CFFCF11DD06E0E9D
:10237000025D01E087D0006B0F0E0115106EC11CCD
:102380000F0B105C01E20083F00E0115066FE850A0
:1023900005E10101960EF26F720E6BD0100E065D14
:1023A0000BE126D9EFCFFCF1EDC1FAF1EEC1FBF163
:1023B00007C9F9F185EF12F0200E065D39E118D951
:1023C000EFCF06F90751081120E1330E03D907506A
:1023D000300F0101DA6F2E0EDB6F330EFBD803C016
:1023E00006F9090103500A0DB8D80101DC6F0A0E85
:1023F000F1D807C006F909010750640DAED80101F4
:10240000DD6FDE6B0901076B086B0751D5D8F8D873
:10241000EF6E0751D1D836E007C910F008C911F0A6
:10242000072B000E082307C9F3FF08C9F4FF1200A9
:10243000300E065D03E1020E001506E1500E065D4A
:1024400008E1020E001505E10101C00EF26F720EE7
:1024500010D0400E065D03E1020E001506E1600E8D
:10246000065D10E1020E00150DE10101C50EF26FCF
:10247000720EF36FEDC1F0F1EEC1F1F107C9EFF1AA
:1024800045EF12F0F368F46812000101EF51F76AAA
:10249000F225F66EF351F7220800F550F0C1E9FF7E
:1024A000F1C1EAFFEF6EF0C1E9FFF1C1EAFFEF50C1
:1024B00003E1F368F4681200EF2BEF51116AEFC1EA
:1024C000F3FF11C0F4FF12000101F451F7250901D7
:1024D0000A6F000E0101F821AA6E0AC9A9FF3F0E7A
:1024E000A616A680A850F5C1E9FFF6C1EAFFEF6E77
:1024F000A85003E1F368F4681200F42BF451116A58
:10250000F4C1F3FF11C0F4FF12000101F95110E111
:10251000DA0EE66E010EE66EFC51E66EE66ADEEC61
:1025200031F0E552E552E552E5520101DF6BF96BFE
:10253000F95142D8FAC1E9FFFBC1EAFFEF6EF95148
:102540003BD803E1F368F4681200F92BF951116AE2
:10255000F9C1F3FF11C0F4FF1200F3CF10F0F4CF74
:1025600011F0330E0B6E0C6AF3CF06F0F4CF07F0C8
:102570009EEC39F006C010F007C011F0300E0624B2
:1025800012000201F06FF16B090116510201EE6FAA
:10259000EF6B000EEE27090EEF23E5EC2BF00009A0
:1025A000120037D8090E05EF13F0EBC1E9FFECC1BB
:1025B000EAFF040E05EF13F0EA6ADA0FE96E010E86
:1025C000EA22EF50120003C9E9FF04C9EAFFEF5005
:1025D00005151200106E0C6E06C907F0C5EF39F034
:1025E000E0C1E9FFE1C1EAFF090E0FD8EF50120088
:1025F0000F0E0115EA6ACA0FE96E020EEA221200F6
:10260000EDC1E9FFEEC1EAFF1200E926000EEA2261
:0C2610001200E7C1E9FFE8C1EAFF120078
:04261C000B01AA6B99
:1026200085C3A4FB86C3A5FB0901036B080E035DEC
:1026300015E2500E01014F6F506B6EEC04F0E66E28
:102640000901E3DB56EC17F0E0DB020EC0DBEF6ABA
:10265000DCDB090EBCDBEF6A032BE8D71200ABCB47
:1026600000F9ACCB01F9090100C9E9FF01C9EAFF92
:10267000002B000E0123EF502E0807E000C9E9FFF0
:1026800001C9EAFFEF50EFE10A0C026B0251106E34
:10269000116A100E105C000E115814E20251A0DBFA
:1026A00000C9E6FF01C9E6FFF8EC35F0136E050E30
:1026B000E15E1350000903E1090102511200090112
:1026C000022BE4D70A0CBFDB04E0200E0901005DF9
:1026D000FAE00901016B2B0E0901005D02E1200EF9
:1026E000006F2F0E005D1FE05C0E005D1CE0200EF1
:1026F000005D1BE03F0E005D18E00D0E005D15E073
:102700000A0E005D12E00C0E015D0DE2610E005D2F
:1027100005E300517A0802E3200E005F0151012B0E
:10272000AADB00C9EFFF8FDBD6E109010151A3DB72
:10273000EF6A090101510CE1E30E106E710E93DB9B
:10274000AECBE6FFAFCBE6FF0EEC36F0050EE15E5A
:102750003F0E0901005D01E1010C000C0B01A451C9
:102760000301855D106E86510B01A555116EE00EBB
:10277000105C2E0E115801E3AA6B0901876B080E3D
:10278000875D06E287C9B0FB04D80901872BF7D71C
:1027900012000B01B0510A0DF3CF7CF9F4CF7DF993
:1027A000540E09017C270B0E7D23010E7A6F09015F
:1027B0007A5101E182D17A6B05DB64DB0AE17CDBD3
:1027C000EF50020B01E0AFDB77DBEF9479DBEF6AD0
:1027D0001200F8DA020EEB50070AE9E0010A01E103
:1027E0005CD1030A01E12DD1010AE1E0070ADFE033
:1027F000010A01E118D1030A01E1D6D0010AD7E1AB
:10280000E1DA4DDBD4E00901010E7A6F85C3A4FB48
:1028100086C3A5FB51DBEF6A6ADB0B01B66FAAD951
:102820000901796F49DBEF9462DB0101916F5DEC87
:102830000CF067DBEE52060ECADA0B01A651EE1859
:1028400020E1A751EE181DE1A851EE181AE1A95197
:10285000EE1817E116E1AA5102E02EDBEF84020E1A
:10286000AA5D02E0000E01D0010E106E25DB1050B3
:10287000010BF36EF346F346F346F70EEF14F31035
:10288000EF6E0901795101E089D00B016C0EAE6F3A
:10289000090EAF6F2CDB0B01AD6F15DF0901806FE7
:1028A000580E6C5D15E108DBEF50040B11E10A0EC8
:1028B000E66EE66AED0E106E710ED5DA6C0EE66EFF
:1028C000090EE66ED5EC35F0136E070EE15E13507F
:1028D0000B016C0EAB6F090EAC6FC1DEE66EEADA6F
:1028E000E5DA090180510BE001016C0EE96F090E78
:1028F000EA6F7CC9E7F17DC9E8F140EC10F018DB24
:10290000DFDA050EEF6EE6DAD1DA00DB106E060EC6
:10291000105C30E312DB04082DE36C0EE66E090E4A
:10292000E66E27EC36F0E552E552F3CF7BF905DB96
:10293000030802E3030E01D0020E09017B5FFDDAFA
:102940000B0FE66EB7DAB2DAF8DA4ADA7B51146ABC
:102950006C0F136E090E142213C0E6FF14C0E6FFBD
:102960000EEC36F0156E050EE15E1550B3DAE55249
:10297000E750EF6ECBDAFF0803E1D3DAEF6A06D057
:10298000C5DAFE0806E1CDDA030EEF6E99DA050E20
:1029900082D092DAEF8294DA010E7DD0790501E0DF
:1029A00006D78EDA030E77D0B5DA01E100D7090138
:1029B000010E7A6F0B016C0EBB6F710EBC6F4EDA9D
:1029C0000B017C0EBB6F710EBC6FA7DA73DAEF34AC
:1029D000EA6AFE0BEA36E96E6E0EE926020EEA227C
:1029E000EECFBBFBEDCFBCFB39DA64DAEFCF10F0F2
:1029F0000B0E105C06E30B018B0EBB6F710EBC6FF0
:102A00008CDAB0CBB9FBA6D998DA060803E154DA20
:102A1000EF8002D051DAEF90D5D9030ED8D9EF6A02
:102A20004FDA020E38D0CED93ADA01E081DA7CC929
:102A3000B7FB7DC9B8FBDCD8000901E1B8D673DA71
:102A400028D068DA01E1B3D66CDAEF34EA6AFE0B1B
:102A5000EA36E96E8E0EE926020EEA22EECF7EF904
:102A6000EDCF7FF909017EC9F6FF7FC9F7FF7E2B05
:102A7000000E7F230800F5CF7BF9F55005E07BC9F8
:102A80005AF1A0D9D1D9EED732DA0101576F75ECDE
:102A900005F016DA060EEF6E8AD694D9F3D90AE05D
:102AA00039DA08E024DA0101566F35EC05F008DA6E
:102AB000070EEF6E01DAEF947AD61200B4CBE9FF7D
:102AC000B5CBEAFFEF0409011E6F1D6BEF6A1F6BA8
:102AD0001E510B01EA6AB225E96EB351EA22EF6A90
:102AE00009011F5141E101011C0E626F090E636F64
:102AF000B1CB61F1B9EC06F0000936E03D0E0901F9
:102B00001C5D0BE11C6B1E511D5D1EE21D29B4CB2B
:102B1000E9FFB5CBEAFFEF6E17D0260E1C5D02E190
:102B2000020E0AD0200E1C5D06E00D0E1C5D03E0B7
:102B30000A0E1C5D04E1010E1F6F1C6B05D02B0EED
:102B40001C5D02E1200E1C6F1E511D5D06E2B2CB22
:102B5000E9FFB3CBEAFF1CC9EFFF0B01B22B000E5C
:102B6000B32309011D2BBCD709011F5101E1000C42
:102B70001F0512000901056B040E055D19E20551E0
:102B80000101626F636B000E6227090E6323B6CBEF
:102B900061F1B9EC06F000090BE009010551052BC4
:102BA000EA6A000FE96E090EEA22EF502008E4E11C
:102BB00009010551EA6A000FE96E090EEA22EF6A7F
:102BC000470E005D07E1450E015D04E1540E025D14
:102BD00001E1000C500E005D0AE14F0E015D07E1BE
:102BE000530E025D04E1540E035D01E1010C020C81
:102BF000F2D813D901E1A6D00901856BECD8030EF8
:102C0000EB50040818E0E7D814D9400B0DE1E3D8E5
:102C1000010EEB500201386F99EC29F00901866F23
:102C2000DAD807D9200B07E0D6D8EF500101576F4B
:102C300075EC05F0010CCFD8090EC9D8EF50010B87
:102C400001E17BD0C8D8030EEB50040A50E0070A1C
:102C500034E0010A1BE0030A0BE0010A6BE1250ED8
:102C6000865D03E131D9010E26D0010E856F62D059
:102C7000250E865D03E1010E856F5AD029D9030E1A
:102C8000A6D886C9EFFF20D9020E15D0610E865D49
:102C900002E3270E04D0410E865D02E3070E865F35
:102CA000300E865D100DF350E66E12D9020E8FD8ED
:102CB000FDD80AD9030EEF6E3DD0610E865D02E3AA
:102CC000270E04D0410E865D02E3070E865F300EAC
:102CD000865D106EFDD8020E7AD81050EF12F4D82F
:102CE000040EEF6E78D873D8EE6AED6A23D0010136
:102CF000860EED6F090EEE6FB7CBEBF1B8CBECF1B2
:102D0000DDEC10F0F3CF10F0F4CF11F0E1D8F3CFF9
:102D1000EEFF11C0EDFF0901010E856FD9D8FF0E3E
:102D2000EE1808E1FF0EED1805E1865101E1856B13
:102D3000CBD8EF6A855101E15BD786C95AF14BD8F0
:102D400073D856D748D8010EEB500201376F72EC9A
:102D500029F0000C0B01B9510A0DF3CF85F9F4CF1E
:102D600086F9540E090185270B0E862301010D0EED
:102D7000C1D801010A0E7AEF17F00B01BA510A0D02
:102D8000F3CF85F9F4CF86F9540E090185270B0E90
:102D90008623BBCBF6FFBCCBF7FF0800F55011E054
:102DA0000B01BBCBF6FFBCCBF7FFBB2B000EBC234C
:102DB0000800F5CF5AF185C9E9FF86C9EAFF34D882
:102DC000E8D712007CC9E9FF7DC9EAFF1200E926B5
:102DD000000EEA221200B7CBE9FFB8CBEAFF1200DF
:102DE000040DF3CFF6FFF4CFF7FF2C0EF626710E8D
:102DF000F722F6CF10F0F7CF11F0126A10C0E6FFFD
:102E000011C0E6FF12C0E6FF120003510A0D79D887
:102E1000540EE9260B0EEA221200EF500101586F02
:102E2000D9EC05F000091200EF500101596FF2EFE3
:102E300005F0010EEB50080D64D8000EE926020ED5
:102E4000EA22EF5012000101000E626F090E636F5B
:102E5000ADCB61F1B9EC06F0000912005ED8B0CB41
:102E6000B9FBAAEF16F0116E126A10C0E6FFE66E0B
:102E700012C0E6FF12000B01EA6AAE25E96EAF51FF
:102E8000EA221200EF500101556F2CEC05F0000909
:102E90001200010EEB500201366F6AEF29F0EF507D
:102EA0000101696F44EC07F000091200E552E75098
:102EB000EF6E120036D844D085DF090EE7EF16F02A
:102EC00081DF020EE7EF16F086DF030EE7EF16F064
:102ED00082DF36D00201356B02016C0E336F090EB2
:102EE000346FCDEC28F0E66E6DDFEE5212006ADF33
:102EF000EF5012005A6F85C9E9FF86C9EAFF14EF47
:102F000017F0F3CFE9FFF4CFEAFF12005BDF010E09
:102F1000EB50120057DF0DEF17F0B0CBBAFBBDEF4F
:102F200016F050DF0DD0C8DFEF924CDF49EF17F0FD
:102F3000DEDF0101606F9BEF06F0BCDFEF50120097
:062F4000040EE7EF16F09D
:0A2F4600966A8688988802014A6B9B
:102F50004B6B4C6B4D6B4E6B4F6B0901006B005113
:102F6000106E116AD890115004E6010E105C000E2C
:102F7000115814E20051040DF3CF10F0F4CF11F00A
:102F8000400E1026000E11220051AFDB10C0EFFFE3
:102F90000051ABDBEE52EF80002BE1D71B6A020140
:102FA000496933DBB7DB02011F0EB1DB0201656F3C
:102FB00002011F0EA9DBAEDB0201210EA0DBAADBA2
:102FC0000201080E656F02010E0EC7DB0A0EC5DB9B
:102FD0000B0ED1DB040E656F02010C0ECCDB020E72
:102FE000656F02010D0E90DBDBDB8EDBB1DB010ECA
:102FF000C2DB600E656F0201020E86DBA9DB030EE9
:10300000BADB65690201070EA8DB0F0EB4DB610EA7
:1030100076DBBCC265F20201010E76DBBDC265F251
:103020000201020E71DBBEC265F20201030E6CDB0F
:10303000BFC265F20201040E67DBC0C265F2020185
:10304000050E62DBC1C265F20201060E5DDB0901FD
:10305000006B080E005D0AE202016569080E0901B5
:103060000025020151DB0901002BF3D771DB070EAC
:103070004BDB440E186E0201220E41DB51DB0D0EBC
:103080007ADBE00E3CDB0201C00E656F0201010E2F
:1030900064DB040E62DB010E6EDB200E7FEF1BF0A3
:1030A00002010D0E70DB02014A2711504B23020171
:1030B0000E0E69DB02014C2711504D2302010F0E49
:1030C00062DB02014E2711504F23120002014951C9
:1030D0001B5C09E10201666BB3DA040B03E1020138
:1030E000496964D3000C62D325DB86A8FED78D8C9A
:1030F0006B0E8D6E836A8D9C86A8FED722DB86A818
:10310000FED78D8C670E8D6E400E836E8D9C86A8CB
:10311000FED78D8C700E8D6E50C283FF8D9C86A85D
:10312000FED78D8C192A000E1A221200020153516B
:10313000541101E11200010E5315106E116A535122
:10314000102409013E6F02015451112009013F6F03
:10315000956A670E8D6E400E836E8D9C86A8FED795
:103160008D8C6A0E8D6E3EC983FF8D9C86A8FED71E
:103170008D8C6B0E8D6E3FC983FF8D9C86A8FED70C
:10318000E0DA86A8FED78D8C0201535119265451DE
:103190001A22700E8D6EE4DA86A8FED78D8C53C28B
:1031A0003CF954C23DF90901010E3C5F000E3D5B44
:1031B00009013CC910F03DC911F03C07000E3D5B10
:1031C0001050111030E0080E3C5D000E3D5926E312
:1031D00089DA86A8FED78D8C85DA86A8FED78D8CF5
:1031E00081DA86A8FED78D8C7DDA86A8FED78D8CF5
:1031F00079DA86A8FED78D8C75DA86A8FED78D8CF5
:1032000071DA86A8FED78D8C6DDA86A8FED78D8CF4
:10321000080E09013C5F000E3D5BD5D763DA86A836
:10322000FED78D8CC5D7120085DA86A8FED78D8C87
:103230006B0E8D6E836A8D9C86A8FED78D8CFF0EDB
:10324000195C1DE15F0E1A5C1AE1090132693369EC
:1032500032C967F233C968F201DA66DA86A8FED7A6
:103260008D8C0201100E53DA0901316F326B440E5E
:10327000336F32C967F2E8CF68F2F0D910D054DA70
:1032800086A8FED78D8C9568700E8D6E8D9A86A857
:10329000FED783CF31F98D8A192A000E1A2209012F
:1032A0003151120057C2B7F958C2B8F9020157514B
:1032B000581103E1F36AF46A1200956A6A0E8D6E82
:1032C000B7C983FF8D9C86A8FED78D8C6B0E8D6E43
:1032D000B8C983FF8D9C86A8FED78D8C25DA86A879
:1032E000FED78D8C0901B7511926B8511A22600EEC
:1032F0001A5C02E31C0E1A5E9568700E8D6E090151
:10330000B7C910F0B8C911F0B707000EB85B10507C
:1033100011100FE08D9A86A8FED7020155C2E9FF71
:1033200056C2EAFF552B000E562383CFEFFF8D8A3E
:10333000E6D757C2F3FF58C2F4FF120002015951F9
:10334000D4D9EE52EF90120002015A51CED9EE526A
:10335000EF805AC21BF0120018C036F90901010EA5
:10336000356FE8CF67F218C068F278D95DDF0901E0
:10337000346FE8CF65F20201030E84EF1BF0FED933
:103380000901006F0201200EBAD918500901005D31
:1033900005E2600ED8801854002502D01850005D58
:1033A000016FE850106E116A1C0ED8801056000E86
:1033B000115610C001F910C003F9026B02C9F3FFE6
:1033C00010C0F4FF12000201E00EE5D90901006F00
:1033D0000201200E94D909010051040B01E0000CF8
:1033E000010C5DC2E9FF5EC2EAFFEF68C7D90901BF
:1033F000126F0201200ECFD90901136FDCD9100B17
:1034000037E00201666B1CD9040B0901176F02013A
:10341000210E75D9020EE66E87EC39F0E55280D99F
:103420000A0E9BD90B0E70D90901175108E0C3D9B8
:103430000A0B02E0000E01D0010E0901176F020114
:10344000020E656F02010D0E96D9220E58D912C9CF
:1034500018F082DF020165690201070E7ED90D0EA8
:1034600053D90901175103E00201260E48D9000C77
:1034700009011351125D67E013C915F9146B14C9E2
:1034800067F213C968F2EAD8120E0201576F586B3F
:103490000201000E556F090E566F04DF090100513D
:1034A000010B4EE0400E025D000E035949E3EE0EA3
:1034B000D8800255050E035543E3600E015D40E2DE
:1034C0000151106E116AD890115004E6440E105C40
:1034D000000E115835E310C9D8F211C9D9F27EECAB
:1034E0002AF0F3CF10F9F4CF11F9060EE66EE66A72
:1034F0000A0EE66E090EE66E5BC2E9FF5CC2EAFFE9
:103500005BC210F05CC211F05BC2E6FF5CC2E6FF7A
:10351000AAEC35F0126E060EE15E1250080E09019B
:10352000115D0BE1105103E0060E105D06E15DC276
:10353000E9FF5EC2EAFF10C9EFFF13C918F0010CE2
:1035400012C918F009DF000C02010A0E656F0201B2
:10355000070EDAD81DD9EFCF41F90901406B40C9F8
:1035600067F241C968F27AD8060E0201536F546BB4
:103570005FC251F260C252F2D9DDBCC250F2B4DD7A
:10358000BDC250F2B1DDBEC250F2AEDDBFC250F2DC
:10359000ABDDC0C250F2A8DDC1C250F2A5DD020110
:1035A000615103E10901426B03D00901060E426F2C
:1035B0000201080E506F98DD42C950F295DD0E0EE3
:1035C00002016227000E63233C0E625D000E635908
:1035D00003E23C0E626F636B62C240F963C241F961
:1035E00062C265F20201050E8FD841C965F202017F
:1035F000060E84EF1BF0D4D8BED8240E80D81BC092
:1036000049F2C6D8EE52EF8012009568600E8D6EBA
:103610008D8C8D8A8D8E966A0A0EE66EDFEC39F0FF
:10362000E55278D88D9E1200600E020164118D6EF5
:1036300065C283FF956A8D9C86A8FED78D8C12008B
:103640009568600E020166118D6E8D9A86A8FED770
:1036500083CF37F98D8A09013751120067C219F0FB
:1036600068C21AF067C265F20201080E4DD868C23E
:1036700065F20201090E84EF1BF00201090E47D822
:103680000901016F0201080E42D8F36E01C9F4FF6F
:10369000120018C023F90901120E226F02016951AC
:1036A0000901222702016A510901232322C967F275
:1036B00023C968F22EEF1BF06BC21BF069D8EFCF65
:1036C0000DF909010E0E0C6F02016C5109010C2756
:1036D00002016D5109010D230CC967F20DC968F291
:1036E0002EEF1BF00201B0EF1BF0E96EEA6AD890F2
:1036F000E936EA36460EE926020EEA221200656F26
:103700000201646B14EF1BF0646F14EF1BF0666F23
:1037100020EF1BF0050EE66E87EC39F0E552120043
:103720000201656B02011200600E8D6E0A0E836E3F
:103730008D9C1200956A6A0E8D6E010E836E8D9CB3
:1037400012008D8C600E8D6E120E836E8D9C120099
:103750000201440E656F02011200D6DF90EF1BF0EC
:1037600051C2E9FF52C2EAFF512B000E5223EF5023
:10377000836E8D9C1200C8DF020112000201600EF0
:10378000BEDFDBEF1BF0C3DF106E116AE8501200E2
:103790001B5075EF1BF0B3DF0201030E87EF1BF028
:1037A000F7DFEFCF65F20201040E1200F1DFEE52F7
:0E37B000EF50010B12000201070E87EF1BF015
:0237BE000901FF
:1037C000006B020E005D07E200513BDB00512DDB78
:1037D000EF90002BF6D712000901000E016F010EC9
:1037E000026F006B020E005D43E2DCDA0C0EC7DAFA
:1037F000CADA126A136A105011101210131032E153
:10380000D1DA0C0E29C1EBFF0D0E2AC1EBFF01012D
:103810002B512C1111E00A0EE66EE66A2BC1E6FF71
:103820002CC1E6FFBFDA01C910F002C911F001C9CD
:10383000E6FF02C9E6FFD8DAB5DA0A0E2DC1EBFFC2
:103840000B0E2EC1EBFFAEDA0E0EEB6A0F0EEB6A1B
:10385000A9DA100EEB6A110EEB6A00C928F1090112
:1038600000511200140E0127000E0223002BBAD7BC
:10387000FF0C01012F5121EF1FF0020E0101305DFD
:1038800004E230C128F166EF18F0000C0101285164
:10389000140DF3CF0AF9F4CF0BF9000E09010A2732
:1038A000010E0B23CADAEE50ED1004E190DA94DA3F
:1038B0008EDA87DA31C150F274EC18F0BEDAEE2AF3
:1038C000EF22BBDAC4DA01E346D8010C010128512A
:1038D000140DF3CF0AF9F4CF0BF9000E09010A27F2
:1038E000010E0B23A6DAEE50ED1004E151DA74DA82
:1038F0004FDA67DA9EDA01013451EE24106E355149
:10390000EE20116ED60ED8801054030E11540AE228
:1039100090DAEECF34F1EFCF35F1D60ED8803457B0
:10392000030E355734C153F235C154F232C151F24E
:1039300033C152F296EC18F07CDA01013451EE26D4
:103940003551ED2276DA83DA01E305D834C1F3FF8D
:1039500035C1F4FF120001012851140DF3CF08F90D
:10396000F4CF09F9000E09010827010E092315DA21
:103970000C0E05DA40DAF3CF00F9F4CF01F90DDAD5
:103980000A0EFDD938DAF3CF02F9F4CF03F905DADC
:103990000E0EF5D9EECF04F9EFCF05F9080E0901A7
:1039A0000427000E0523066B076B140E02016C6FD3
:1039B0006D6BF3D906DA04C96EF305C96FF3030121
:1039C000110E6D6FEAD908C96BF309C96CF3E9EC04
:1039D0002CF004C9D8F205C9D9F27EEC2AF0F3CF55
:1039E00004F9F4CF05F9080E0201536F546B02017C
:1039F000000E516F090E526F96EC18F0FBEC1AF0A6
:103A0000CCD9120EBCD9EF68C8D90E0EEB6A0F0ED6
:103A1000EB6A1200020E0101365D0AE236C128F19E
:103A2000FFD9D880EE54000EED5401E3000C010CD8
:103A3000000C17DA01E1000C2851F7D9EF50010B07
:103A400001E013DA14EC19F037C1E9FF38C1EAFFDD
:103A5000EF6E11DAEE06EF5AE3D9EE50ED1002E107
:103A6000ACEC19F0010CFDD903E1F36AF46A120021
:103A70002851DBD9EF50010B01E0F7D9FCD983D9EC
:103A80003B51105C3C51115805E2CAD9EECF3BF1D5
:103A9000EDCF3CF13BC157F23CC158F239C155F270
:103AA0003AC156F252EC19F0F3CF00F9F4CF01F914
:103AB000E2D909010051EE5E0151ED5AD2D902E17D
:103AC000ACEC19F03BC1F3FF3CC1F4FF1200C9D9C3
:103AD00002E0ACEC19F0CFD9EE6AED6A1200080EE4
:103AE0000201576F586B0201460E556F090E566F53
:103AF00052EC19F046C95DF947C946F95DC947F965
:103B000048C95DF949C948F95DC949F9080E106EFF
:103B100009014B51D880105403E24A055D6F02D071
:103B20004AC95DF9080E4B5D4A6F5DC94BF94CC936
:103B30005DF94DC94CF95DC94DF93DC1E9FF3EC183
:103B4000EAFF060E1CD9EECF4FF9EECF50F9EECFBB
:103B500051F9EFCF52F955D9EFCF53F9010E0FD9E3
:103B6000EFCF54F94ED9020E0AD9EFCF55F949D902
:103B7000030E05D9EFCF56F9576B110E586F41C19F
:103B800059F942C15AF941C1D8F242C1D9F27EEC89
:103B90002AF0F3CF59F9F4CF5AF90C0E0201E06F75
:103BA000E16B02014F0EDE6F090EDF6FB2EC2AF0FF
:103BB000F3CF5BF9F4CF5CF909015B1F5C1F1A0EB0
:103BC000FBD85BC950F274EC18F05CC950F274EC8D
:103BD00018F0140EF1D841C1E2F242C1E3F20EEC4A
:103BE0002BF0F3CF5BF9F4CF5CF909014C51F318DA
:103BF00016E14D515C1913E13FC147F140C148F155
:103C00003DC145F13EC146F10101460E436F090E2B
:103C1000446F1CD809014E6FFF0E4E5D03E1ACEC02
:103C200019F0010C4E51A1D8100EA9D84AC9EEFFC7
:103C30004BC9EDFF4E51F9D8EF80010C010128511D
:103C400094D8E9CFF3FFEACFF4FF1200090101692C
:103C5000000E026F010E036F006B020E005D5BE24F
:103C6000A6D80C0EFAD8020E8AD8D5D80001125068
:103C700010184AE11350111847E199D80A0EEDD8EF
:103C8000CAD8125010183EE1135011183BE18FD8DA
:103C9000100E75D8EECF14F0EFCF15F0166A176A34
:103CA00014501510161017102DE145C1E9FF46C13B
:103CB000EAFF060E64D8EECF10F0EECF11F0ABD8CD
:103CC00076D8060E5CD8EE50101808E1EE501118A8
:103CD00005E1EE50121802E1EE50131810E047C152
:103CE000E9FF48C1EAFFE868EE180CE1E868EE1861
:103CF00009E1E868EE1806E1E868EE1803E1090159
:103D00000051120000C901F90901140E0227000E2A
:103D10000323002BA2D7FF0E015D24E00151140DF7
:103D2000F3CF02F9F4CF03F9000E0227010E0323AB
:103D30000A0EE66EE66A45C1E6FF46C1E6FF37D8E1
:103D400002C910F003C911F002C9E6FF03C9E6FF7A
:103D50004BD85CD818D82BD80A0E10C0EBFF0B0E2E
:103D600011C0EBFF090101511200140DF3CFE9FF5F
:103D7000F4CFEAFF000EE926010EEA221200E9263E
:103D8000000EEA221200EECF10F0EFCF11F0120079
:103D90000AC9E9FF0BC9EAFF120008C9E9FF09C90E
:103DA000EAFF120001C9E9FF02C9EAFF120002C9D5
:103DB000E9FF03C9EAFF12000201696F6A6B49EF6C
:103DC0001BF0120EEB5002016B6F5CEF1BF00AC987
:103DD000E9FF0BC9EAFF1200120E1BC0EBFF1C0E1D
:103DE00002016C6F6D6B1200AAEC35F0126E060EBC
:103DF000E15E12501200EECFD8F2EDCFD9F27EEF95
:103E00002AF03FC1E9FF40C1EAFF120043C1E9FFC8
:103E100044C1EAFF1200EECF12F0EFCF13F0120010
:103E20002851A3DF100EBFEF1EF09FDF130EBFEF70
:103E30001EF0AEDF0E0EBFEF1EF0C9DF0E0EBFEF9D
:103E40001EF093DF0C0E9BDFEE6AED6A12009BDF23
:103E5000D60E105C030E1158120091DF94DF06EFAE
:103E60001FF009D8EE50ED1012002851DEDFEF9060
:0C3E70001C0EDCEF1EF0010110EF1FF033
:043E7C00070E030129
:103E8000905D01E11200FF0E915D01E0A7DA0301F0
:103E90009169906B936B120003019051060A01E146
:103EA000A2D0030A66E0010A59E0070A46E0010AC7
:103EB00033E0030A27E0010A01E0120009010E695C
:103EC0000F69106911691269136914691569166916
:103ED00017690301086B096B0A6B0B6B430E010139
:103EE0002D6F2E6B01010E0E2B6F090E2C6F440EE1
:103EF0000101296F2A6BECEC1BF00301916F62DA70
:103F0000010E906F50DA140E105C000E115801E291
:103F10007DD00301020E3BD00301085109110A11A3
:103F20000B1133E191C330F13DEC1CF000096EE060
:103F30000301010E5FDA030E2AD061DA03E3030105
:103F4000020E906F91C336F10AEC1DF000095EE09D
:103F500063D802085BE10301040E906F91C330F156
:103F60003DEC1CF0000952E00301030E43DA050E9C
:103F70000ED091C336F10AEC1DF000092EE04CD8AA
:103F80000901186F060E185D04E10301040E906F1D
:103F90001200050E185D26E121DA0301916912DA9B
:103FA000060E906F08C3B8F209C3B9F20AC3BAF299
:103FB0000BC3BBF210C3C2F211C3C3F212C3C4F2EB
:103FC00013C3C5F20CC3C6F20DC3C7F20EC3C8F2C9
:103FD0000FC3C9F29281932B120011DA17E3030188
:103FE000020E906F1200DFD9640E105C000E1158A3
:103FF0000DE30407000E055B065B075B045105112A
:104000000611071102E10301906BDCD912000301D4
:10401000080E906FEEEF21F00901026B03013C0ED8
:10402000046F056B066B076BB0D9020E0901005DCA
:1040300001E0EBD0016B0F0E015D02E2EFD9FBD77F
:104040000101080E376F030EABD9090E376F030E4F
:10405000A7D90A0E376F030EA3D90B0E376F030EC5
:10406000C6D90901016B080E015D02E2D7D9FBD761
:10407000BCC208F9BDC209F9BEC20AF9BFC20BF938
:10408000C0C20CF9C1C20DF9016B060E015D0EE252
:104090007CD909010151EA6A080FE96E090EEA228A
:1040A000EF50005D01E0D3D0012BEFD7016B015140
:1040B000106E116AD890115004E6CE0E105C000EFE
:1040C000115802E2ABD9F3D7036B5FD90901005154
:1040D000330A62E0CC0A5DE0C90A47E0350A23E012
:1040E000020A0DE0340A01E07DD04FD90901000534
:1040F00001E0ADD00101020E376F090E48D072D930
:1041000001E0A5D00101100E376F030E49D9110E41
:10411000376F030E45D9120E376F030E41D9130EB8
:10412000376F030E34D05ED901E291D001010C0E3D
:10413000376F030E35D90D0E376F030E31D90E0EC2
:10414000376F030E2DD90F0E376F030E50D9040EA3
:104150000901005F090100510007000952E0010157
:10416000010E376F090E43D9F5D73CD970E1010133
:10417000070E376F090E14D9060E376F090E10D9C6
:10418000050E376F090E0CD9040E376F090E2FD9A3
:1041900038D0010E036F35D025D959E10101070E42
:1041A000376F030EFDD8060E376F030EF9D8050ED4
:1041B000376F030EF5D8040E376F030E18D9D88069
:1041C000080E03010455070E0555000E0655000E96
:1041D000075517E2080E045F070E055B000E065B2D
:1041E000075B0FD00101000E376F090E00D90901DE
:1041F00000510007000905E00101010E376F090EAB
:10420000F5D70901035101E160D7020E025D09E112
:1042100004C900F305C901F306C902F307C903F392
:1042200011D0000EE96E030EEA6EEE50041908E19B
:10423000EE50051905E1EE50061902E1EE5007199E
:1042400001E0026B67EC1DF009010251120067ECFE
:104250001DF0000C0101010E9ED8010E9CD8060E27
:104260009AD8ABD8120E97D8230E95D8340E93D87F
:10427000560ECBD8800EC9D8A0D89FD8316B46EC4B
:104280001CF00901196B0C0E195D02E2A0D8FBD7D6
:10429000BCC231F146EC1CF0BDC231F146EC1CF061
:1042A000BEC231F146EC1CF0BFC231F146EC1CF04D
:1042B000C0C231F146EC1CF0C1C231F146EC1CF039
:1042C0000901196B1951106E116AD890115004E64A
:1042D000CA0E105C000E115802E279D8F3D7010122
:1042E000630E59D8820E57D8530E55D8630E53D843
:1042F000350E51D8010E316F46EC1CF016C331F16A
:1043000046EC1CF00301160518E0085109110A11CA
:104310000B1113E00101360E7CD803C331F146ECDA
:104320001CF002C331F146EC1CF001C331F146EC44
:104330001CF000C331F146EC1CF00101370E2BD804
:10434000020E29D8010E27D8030E316F46EC1CF05F
:10435000030E0301165D13E10101320E5AD808C3A2
:1043600031F146EC1CF009C331F146EC1CF00AC3F4
:1043700031F146EC1CF00BC331F146EC1CF00101AD
:10438000316946EC1CF0ABEF1CF00101000E376FF9
:10439000090EF7EF21F0316F46EC1CF0010112001D
:1043A00026D801011200030114510301855D106E2E
:1043B000865103011555116E1200316B46EC1CF04D
:1043C0000101120085C314F386C315F31200010125
:1043D000316B46EC1CF00901192B120091C32FF12F
:1043E00039EF1CF0D2DF040E0901005D1200386FB6
:1043F00019EF1DF0166F2EDFE5DF03011200D3DF8A
:10440000900E105CFF0E11581200C5DFD6DFDDEFF5
:1044100021F0C1DF040E316F46EF1CF0B6DF090159
:04442000012B12005A
:0C4424000001F35101E112000001110E33
:10443000F16F690EF26FECEC37F00001210EF16FB5
:10444000670EF26FECEC37F0F3C0B6F90901B65124
:10445000000814E2B651070B05E100012E0EED6FC6
:104460008DEC37F027DA02E057D908D0320EE66E2D
:1044700087EC39F0E5520901B607E8D75FEF24F081
:104480003CDAE7D9010EE926000EEA22E2D9020E53
:10449000E926000EEA22DDD9030EE926000EEA2203
:1044A00070EF24F00901016B05DAFEE07DEC37F0D6
:1044B0000901006F0D0E005D17E00A0E005D14E0AB
:1044C000012B0001F6C0E9FFF7C0EAFFF62B000E52
:1044D000F72300C9EFFFF6C0E9FFF7C0EAFFEF6A74
:1044E000F851F8070009E0E1090101511200F9C093
:1044F00001F9FAC002F90901036BF9C0E9FFFAC03A
:10450000EAFFEFCF00F9EF5021E02E0E0901005D28
:1045100011E10001F9C0E9FFFAC0EAFFF92B000E32
:10452000FA23EF6AAFD9032BD1D9F9C001F9FAC048
:1045300002F907D0300E005D03E30051390801E2B3
:10454000000C0001F92B000EFA23D7D79BD9BED956
:10455000030E0901035D01E0000C010CABD9FEE084
:104560007DEC37F00901006F310E005D05E3390E77
:10457000005D02E200511200390CA1D9300E000199
:10458000FD5DFF0FE96EEA6AD890E936EA36440E1F
:10459000E926030EEA22EECFF1F0EDCFF2F0ECECDB
:1045A00037F00001FD51380A01E1B5D00F0A01E1F1
:1045B000B0D0010A01E1A1D0030A01E197D0010ABC
:1045C00054E0070A4BE0010A42E0030A01E012004E
:1045D0000201330ED66F96EC36F00901A16F02018D
:1045E000340ED66F96EC36F00901A26F870EE66E98
:1045F000090EE66EA1C9E6FFA2C9E6FF87D9870EBC
:10460000EF6F090EF06FDBEC37F029D9000947E0B6
:10461000870EE66E090EE66E69EC31F0E552E55262
:10462000F3CFA1F9F4CFA2F9F3CFA8FF0201330E23
:10463000D76FA0EC36F0A2C9A8FF0201340ED76FE5
:10464000A0EC36F0A2C9C0F2A1C9C1F21200090162
:10465000B80E9F6F020EA06FA36B0ED00901C60E9D
:104660009F6F020EA06F0E0E06D00901C20E9F6F43
:10467000020EA06F0A0EA36F9FC9F4F0A0C9F5F057
:10468000FFDEEDD800019B0EFB6F090EFC6F0001F1
:10469000870EF96F090EFA6F2ADF00090BE100019E
:1046A000C70EF16F680EF26FECEC37F003D9FEE045
:1046B0007DEF37F09FC9E9FFA0C9EAFF9BC9EEFF74
:1046C0009CC9EEFF9DC9EEFF9EC9EEFF9BC9A8FFE6
:1046D000EAD89CC9A8FFE7D89DC9A8FFE4D89EC91D
:1046E000A8FF0901A351A32B020110D00201160E4D
:1046F000D66F96EC36F0010906D00201160ED66F81
:1047000096EC36F0FE0BA86E0201160ED76FA0EFE6
:1047100036F0A1EF23F0120000015A0EF16F670E80
:10472000F26FECEC37F01ADF0901B76F390EB75DA5
:1047300003E0B7C9FDF021DF380E0901B75DECE1F8
:1047400012000901006B026B02EC2AF085C385F9A7
:1047500086C386F9090185510301855D106E865176
:1047600009018655116E320E105C000E115809E3D6
:1047700085C385F986C386F90001150EED6F8DECB2
:1047800037F098D8E7E00901025162E193D8FBE0E5
:104790007DEC37F00901016F0051030A20E0010AA6
:1047A0001BE0030A14E0010502E1010E16D0040E1D
:1047B000015D09E14BEC2AF00001060E9BD80901CE
:1047C000010E026FE0D70001150E94D8DCD7060E5B
:1047D000046F036B020E01D0030E006FD4D7035198
:1047E000032BEA6A050FE96E090EEA2201C9EFFF01
:1047F0000351106E116A1134C6E210508008000E89
:104800001154C1E2060E046F016B0151106E116A62
:10481000D890115004E6800E105C000E11580DE285
:104820000151EA6A050FE96E090EEA22EFCF45F25F
:104830001AEC2AF00901012BE8D70201376B72EC60
:1048400029F004C9EDF08DEC37F00901006B9BD71E
:10485000010C46D800012E0E4DD87DEF24F000014A
:10486000290E48D800013A0E45D80001200E42D842
:104870000001140EF86F0001870EF66F090EF76F36
:1048800052EF22F001C9E6FF02C9E6FF69EC31F000
:10489000E552E552F350E66EFBC010F0FCC011F09B
:1048A0000901035112000901A351A32B0201D76F83
:1048B000A0EF36F00001EA510001EB5D12000001AB
:1048C0000D0E18D800010A0E7AEF24F00F01102403
:1048D000E96E000E1120EA6EE552E750EF6E12000D
:1048E000EF50E66EE66A12D8000EEF6F090EF06F19
:1048F000DBEF37F0ED6F8DEF37F0000EE66E090E4F
:10490000E66EF4C0E9FFF5C0EAFF1200DEEC31F01C
:0C491000E552E552E552E55200011200AC
:04491C00150E010172
:104920004F6F506B6EEC04F00101936F976BC56B8A
:10493000926B140E956F966B120093C155F12CEC8F
:1049400005F0000907E10101C56B070E996F976B30
:10495000926BA6D093C169F144EC07F0000934E0F2
:1049600020DA0101700E626F090E636F93C161F16D
:10497000B9EC06F000090EE01F0E0101C55DF1E281
:10498000C551C52BEA6AA40FE96E010EEA2270C96F
:10499000EFFFE7D793C160F19BEC06F00A0E090127
:1049A000705D26E10101C551EA6AA40FE96E010EAE
:1049B000EA22EF6AC56B9BD9C6C1D8F1C7C1D9F14C
:1049C0005DD90101996F14D00101975111E0D551C2
:1049D0000301855D106E86510101D655116E500E92
:1049E000105C460E115804E3DCD9020E996F976FE4
:1049F00001019751020A3EE0070A0DE0040A06E0B1
:104A0000010A54E19A6BCDD9010E976FBED94EE0E1
:104A10000101050E976FB9D92DE09AC1E9FFEA6A45
:104A2000E9BEEA68D890E936EA36A20EE926020E17
:104A3000EA22EECF71F9EDCF72F9090171C9F6FFE3
:104A400072C9F7FF712B000E72230800F5CF70F9C1
:104A5000F55007E070C95AF193C159F1F2EC05F035
:104A6000ECD793C157F175EC05F001010B0E9A6F6D
:104A7000020E976F070E0101995D18E099C1D7F1F9
:104A800016D800090FE00B0E01019A5D02E0050E39
:104A900004D0020E995D02E1010E976F070E996F27
:104AA000986B010C0B0E01019A5DB3E1010C010141
:104AB000D751050A51E0060A4DE0070A34E0060A1C
:104AC00030E0030A18E0010A51E192819293010E4D
:104AD0009A6F090EE66EE66AC8C1E6FFC9C1E6FF35
:104AE0009B0EE66E010EE66E35EC36F0106E060E8D
:104AF000E15E1050010C92A112D0C8C1FEF2C9C1F2
:104B0000FFF202019B0EFC6F010EFD6F84EC28F09A
:104B1000000904E001019283020E29D00101060E72
:104B200026D0B9EF25F0D0C1E6FFD1C1E6FF69EC90
:104B300031F0E552E552F3CF96F1D2C1E6FFD3C191
:104B4000E6FF69EC31F0E552E552F3CF95F1010152
:104B50000A0E0DD0E2EF25F00A0E9A6FFE0E945D5C
:104B600007E094C156F135EC05F0010C050E9A6F83
:104B7000010C01019851030A18E0020A0FE0010A32
:104B800020E1020E985D02E14BEC2AF0FE0E0101DD
:104B9000945D06E010D90101010E05D0FCD811E1A9
:104BA0000101030E9A6F986F000CEFD80AE093C1D1
:104BB00055F12CEC05F0000904E093C156F135ECF9
:104BC00005F0000C01019851020A2EE0030A21E0D1
:104BD000010A53E192B302D0060E4DD0070E9A6F30
:104BE00095C153F196C154F19351220DF3CFE9FFD2
:104BF000F4CFEAFF000EE9260A0EEA22EE52E9CFD0
:104C000051F1EACF52F1AAEC04F00101946F010EC8
:104C100009D0C1D832E0020131A12FD002EC2AF034
:104C20000101020E986F000C94C169F144EC07F089
:104C300000091AE0B6D80101730E626F090E636FA6
:104C400094C161F1B9EC06F0000905E073C945F2C1
:104C50001AEC2AF0F0D70201376B72EC29F094C1FC
:104C600060F19BEC06F0000C96D807E1A4D8010196
:104C7000FE0E946F090E9A6F010C000C0901006B77
:104C8000060EE76E0019E8AE02D0E73402D0E75016
:104C9000005D2CE2040EE66EE66A00C9E9FFEA6AEE
:104CA000E9BEEA68D890E936EA36960EE926020EA1
:104CB000EA22EECF10F0EFCF11F0126A10C0E6FF3B
:104CC00011C0E6FF12C0E6FFD8C1E6FFD9C1E6FF7A
:104CD0008BEC35F0136E070EE15E1350000903E113
:104CE0000901005112000901002BCAD7060C090165
:104CF000036BA40E006F010E016F58D8EF5020080F
:104D000004E1002B000E0123F8D700C9C6F101C948
:104D1000C7F10101010ED46F49D8EFCF02F9EF506E
:104D200033E009010351010A16E0010A29E1200ECE
:104D3000025D03E02C0E025D05E138D8EF6A010E3A
:104D4000036F1ED00D0E025D03E00A0E025D18E136
:104D50002DD8EF6A15D0200E025D12E00101D4516A
:104D6000D42BE96EEA6AD890E936EA36C60EE9260F
:104D7000010EEA2200C9EEFF01C9EDFF0901036B34
:104D8000002B000E0123C8D7120093C158F1D9ECB3
:104D900005F00009120094C155F12CEC05F0000952
:104DA000120085C3D5F186C3D6F1120000C9E9FF10
:104DB00001C9EAFF12004BEC2AF094C156F135EF1D
:024DC00005F0FC
:0E4DC200DACFE4FFE2CFDAFFE9CFE4FFEACF79
:104DD000E4FFF6CFE4FFF7CFE4FFF5CFE4FFF3CF36
:104DE000E4FFF4CFE4FFFACFE4FF00EE00F0100E92
:104DF000E80403E3EECFE4FFFBD700EE10F0080E6B
:104E0000E80403E3EECFE4FFFBD7E652F2A414D0AC
:104E10009E0ED76E580ED66E0301852B000E86238C
:104E20008723882303018B0706E1640E8B6F030140
:104E3000892B000E8A23F2949E50200B05E09D5092
:104E4000200B02E050EC37F09E50100B05E09D5017
:104E5000100B02E066EC37F0E55200EE17F0080E9A
:104E6000E80403E3E5CFEDFFFBD700EE0FF0100EF3
:104E7000E80403E3E5CFEDFFFBD7E5CFFAFFE5CF8D
:104E8000F4FFE5CFF3FFE5CFF5FFE5CFF7FFE5CF83
:104E9000F6FFE5CFEAFFE5CFE9FFE5CFDAFF110046
:104EA0000901800E056F829482920201F751090177
:104EB000051502E0828001D082908282050504E01F
:104EC00005417F0B056FF0D7829212000901266B16
:104ED000276B050E27AF02D0D89003D0265D000EB9
:104EE00027591AE2010E26C9E7FFE75204E0E84617
:104EF000FE0BE706FCE10201F81509E026C9E9FF0F
:104F000027C9EAFF20D9F9C2EEFFFAC2EDFF090175
:104F1000262B000E2723DDD712000901026B036B3D
:104F2000046B006B016B050E01AF02D0D89003D06B
:104F3000005D000E015930E200C9E9FF01C9EAFF36
:104F400011D926E210500008000E115421E200C9C8
:104F5000E9FF01C9EAFFD890E936EA36220EE926D0
:104F6000030EEA22EF50106E010E105204E0E846E4
:104F7000FE0B1006FCE109010313010E00C9E7FF57
:104F8000E75204E0E846FE0BE706FCE109010413E2
:104F9000002B000E0123C7D7038103C9F7F280DF7E
:104FA00002C9F7F27DDF04C9F7F27ADF82848294C6
:104FB0001200C4D8B4EC39F0B9EC28F05EEC0EF075
:104FC0003CEC37F078EC36F0B4EC36F045EC37F0EA
:104FD00003EC37F01AEC37F02FEC37F00201140E27
:104FE000D66F96EC36F00001F36F12EC22F04FEC26
:104FF00030F00EEC13F08EEC24F00201160ED66F9A
:1050000096EC36F0010B06E10301010E176F030168
:10501000070E906F949094929494020E0201F96F8F
:10502000FA6B02011F0EF86F51DF77DF949A829AB4
:105030000201150ED66F96EC36F0020B0CE0030160
:105040002C510301855D106E320E105C04E385C3A4
:105050002CF3939C8A7C03012D510301855D106E16
:10506000640E105C26E385C32DF30901AF6BB06BB2
:10507000050EB0AF02D0D89003D0AF5D000EB0598E
:1050800017E2AFC9E9FFB0C9EAFF6CD80DE21050D2
:105090000008000E115408E2AFC9E9FFB0C9EAFFE9
:1050A00052D8EE06000EEF5AAF2B000EB023E0D719
:1050B00034DF5AEC30F0AEEC13F09DEC24F008D85D
:1050C000030117510301935DB3E093C317F3B0D706
:1050D0000201FB2B0C0EFB5D01E3FB6BC11C0F0BF4
:1050E000FB5D0FE2C30EC216FB51040DF350C2125A
:1050F000C280C282C2B2FED702012DD8C4CFEFFF58
:10510000120029D8EF6A1200350E0201F06FF16B20
:10511000FCC2EEF2FDC2EFF2E5EC2BF000090DE16E
:105120003E0E0201F06FF16BFEC2EEF2FFC2EFF233
:10513000E5EC2BF0000901E1010C000CF18ED56AC1
:10514000F28EF28C1200D890E936EA36180EE92673
:10515000030EEA221200FB51EA6ACA0FE96E020E40
:10516000EA221200F0DFEECF10F0EFCF11F0113491
:0251700012002B
:0E5172000201306B010E316F0301180E546FF5
:105180008BEC34F00901006B060E005D05E2005166
:1051900091D9EF6A002BF8D7010C0901FE0E026FBE
:1051A000020131A1FE0C0901016B060E015D0AE24C
:1051B000015180D9EF50010B03E101C902F902D07E
:1051C000012BF3D7FE0E025D01E1FE0C450E036FCD
:1051D000046B056B33C2E9FF34C2EAFFEF5001E113
:1051E000FF0C33C2E6FF34C2E6FF63EC36F0E55253
:1051F000E552F3CF33F2F4CF34F203C959F304C9C3
:105200005AF367D904E00901FE0E026F5ED015EC77
:1052100035F00901006F00AF02D0026956D0016B72
:105220000C0E015D21E215EC35F00901006F015112
:105230000201EA6A3325E96E3451EA22EF5009018E
:10524000005D06E0120E0327000E042305230CD098
:10525000005108E10901012B0C0E015D05E215EC7E
:1052600035F0F8D7012BDCD70C0E015D2BE1025194
:10527000080DF3CF06F9F4CF07F9000E0627020E4A
:10528000072333D9010EEF6E30D9EB6A020EEB6AB9
:1052900015EC35F0E66E29D9030E03D9030E2AD991
:1052A000010EFFD8030E26D9020EFBD8060EF9D840
:1052B000060E20D9010E1ED9E552E750EF6E02010D
:1052C000302B03D01FEC35F098D71FEC35F00901D7
:1052D0000251120036C237F205D802013651EAD81F
:1052E000EF6A120002013751080DF3CFB1F9F4CF84
:1052F000B2F9000E0901B127020EB223F1D8EF5026
:10530000020B03E01FEC35F00DD0EAD8EF50040B90
:1053100009E00BEC35F00301A00E626F5AEC35F09A
:105320000009F9E1F90EDCD8E850EF1602013193DB
:10533000120002013851080DF3CF01F9F4CF02F940
:10534000000E09010127020E02239F0E106EBCD829
:10535000E850EF16B9D8EF50010B25E0B5D8EF5063
:10536000020B24E1020131B31ED0AED8EE52EECFD3
:1053700013F0EFCF14F0156AA7D8030EBBD8EE5088
:105380001324106EEE501420116EEE501520126E84
:1053900010C059F311C05AF39CD805E195D8EF829B
:1053A0000201318303D090D8EF8A000C15EC35F060
:1053B0000901006F89D8EE52EE2A000EED22EECFE1
:1053C00010F0EDCF11F080D8060E94D8EECF12F089
:1053D000EFCF13F000011250101805E1135011180F
:1053E00002E172D8EF8C090100511200010C010C8E
:1053F00012001200F36AF46A1200056A066A076A6C
:105400001200000C020131A1000C0901B16B060E63
:10541000B15D08E2B1514ED8EF50010B01E0000C34
:10542000B12BF5D70201010E006F400E036F046B24
:10543000056B010C0901000EB36F020EB46F02017F
:1054400000A506D0400E325D03E30201376B4ADF50
:10545000020100B515D031A302D0008B000C03C2AD
:1054600056F304C257F30301A00E556F94EC34F0C9
:10547000000905E1020100853183326B01D0000C87
:1054800045C25BF3F7EC34F00201322B032B000E24
:1054900004230523010C0201376B24DF0201006B9A
:1054A000010C28D8E552E750EF6E15EC35F0E66EAA
:1054B00075EF2AF0080DF3CFE9FFF4CFEAFF000EF5
:1054C000E926020EEA22120001C9E9FF02C9EAFF39
:1054D00012000301A00E586FCAEC34F0000912004C
:1054E000B1C9E9FFB2C9EAFF120006C9E9FF07C95D
:0C54F000EAFF1200E926000EEA2212007A
:0454FC00D9C2F3FF1F
:10550000D8C2F4FF1200DAC201F9DBC202F9DCC230
:1055100003F9DDC204F90901010E056F090E066FDA
:1055200005C9E9FFEA6E030E9AD9EF50E66E030E45
:1055300090D900C9EFFF84D9020E91D9010E85D907
:10554000EF50E66E7DD9020E84D9010E7ED900C9D6
:10555000EFFF01C904F002C905F003C906F004C950
:1055600007F012000901406B416B426B436BDEC2D6
:105570003EF9DFC23FF9E0C23CF9E1C23DF9D89003
:105580003D333C333CC910F03DC911F03C07000EDF
:105590003D5B1050111018E03EC9E9FF3FC9EAFF1A
:1055A000020E3E27000E3F23EECF10F0EFCF11F09A
:1055B0000001105009014027000111500901412349
:1055C000000E42234323DED70201E051010B0EE01F
:1055D0003EC9E9FF3FC9EAFFEFCF10F000011050CC
:1055E00009014027000E4123422343230901425170
:1055F000431109E040514225406F41514321416F21
:10560000426B436BF3D740C910F041C911F0101E33
:10561000111E10C0F3FF11C0F4FF12000901010EAA
:10562000006F016B026B0201E251E3114EE0400E8C
:10563000E25D000EE35904E3400E106E116A04D0DF
:10564000E2C210F0E3C211F010C005F909011050D8
:105650000201576F586B0201060E556F090E566F07
:1056600052EC19F009010551106E116A1050020137
:10567000E25F1150E35B0901046B0551045DD3E265
:105680000451EA6A060FE96E090EEA22EFCF03F928
:1056900000510AE103510125016F0351015D0DE243
:1056A000022B0BE1012B09D003510225026F03519C
:1056B000025D03E2012B01E1022B005102E0000E2A
:1056C00001D0010E006F042BD8D70901021D026F13
:1056D000011DF36E02C9F4FF12000201E451390802
:1056E00005E3300EE45D02E3300E0FD0E4514608CE
:1056F00005E3410EE45D02E3370E07D0E45166088E
:1057000006E3610EE45D03E3570EE45D1200FF0C57
:10571000010E0201EA6AE525E96EE651EA22EFCFC1
:10572000E4F2DBDF0901266FE5C2E9FFE6C2EAFF2A
:10573000EFCFE4F2D2DF0901276FFF0E265D03E011
:10574000FF0E275D01E1000C2739F00B2611E7C29F
:10575000E9FFE8C2EAFFEF6E010C0901266BA6B271
:10576000FED72F0EA616A6840201EBC2E9FFECC2FB
:10577000EAFFEB2B000EEC23EF50A86E0901262B5D
:105780000201ED510901D880265501E2A86AEAC25A
:1057900010F0116A1050AA6E0201E9C210F0EAC2BC
:1057A00011F0E92B000EEA231050A96E550EA76EDA
:1057B000AA0EA76EA6820000A6B2FED7A850D4E11A
:1057C000A6940901265100D01200F1C210F0105029
:1057D000AA6EF0C2A9FF3F0EA6160201EEC2E9FFB3
:1057E000EFC2EAFFEE2B000EEF23EFCF1CF9A680ED
:1057F000A85009011C5D01E0010C1C5101E1000CE5
:10580000A92AEBE1AA2AE9D7F2C202F9F3C203F905
:105810000901006B016B0201F4510901005D0201F5
:10582000F551090101590BE202C9E9FF03C9EAFF79
:10583000022B000E0323EF6A002B0123ECD712008A
:1058400005C9E9FF06C9EAFF1200E926000EEA22AF
:105850001200FBDFE552E750EF6E20EF2CF0F5DF92
:08586000EFCF00F920EF2CF05E
:08586800140E0201576F586B8A
:105870000201080E556F090E566F52EC19F0F00E2A
:1058800009010815400801E0A1D00F0E0815040D0C
:10589000F350106E116A140E105E000E115A10C0F3
:1058A0001CF91050140801E291D01C5100080BE2C1
:1058B0001C510201576F586B02011D0E556F090EE6
:1058C000566F52EC19F012C900F913C901F9090118
:1058D000126B136B140E16D9080EDE6F090EDF6FF4
:1058E000B2EC2AF0F3CF04F9F4CF05F90901041F53
:1058F000051F1C51000810E21C5104D91D0EDE6F5B
:10590000090EDF6FB2EC2AF0F3CF06F9F4CF07F9F6
:105910000901061F071F02D0066B076B040EF2D8A1
:10592000040EDE6F090EDF6FB2EC2AF0F3CF02F93E
:10593000F4CF03F90301080E706F090E716FB5D82B
:1059400009010251001942E1035101193FE1F00E32
:10595000081540083BE10301635164110CE063C387
:10596000E9FF64C3EAFF18C9EEFF19C9EEFF1AC9BF
:10597000EEFF1BC9EEFF65C3E9FF66C3EAFF060E33
:10598000DBD814C9EEFF15C9EEFF16C9EEFF17C923
:10599000EEFF67C3E9FF68C3EAFF11C9EFFF090122
:1059A0001C51126E136A12500A5D106E13500B597F
:1059B000116E140E105E000E115A69C3E9FF6AC31E
:1059C000EAFF10C0EEFF11C0EDFF010CACEC19F0C6
:1059D000000C0901450E286F296B140E03016E257A
:1059E00009012A6F000E03016F2109012B6F0001CD
:1059F000FE2B000EFF23FEC02CF9FFC02DF909017C
:105A00002E6B400E2F6F640E306F6DC331F9326B09
:105A1000336BB8C234F9B9C235F9BAC236F9BBC270
:105A200037F96BC3E9FF6CC3EAFF060E85D8EECFEA
:105A300038F9EECF39F9EECF3AF9EFCF3BF9030160
:105A4000280E706F090E716F30D8140E5BD8280EB7
:105A5000DE6F090EDF6FB2EC2AF0F3CF32F9F4CF2C
:105A600033F9140E03016E250201626F000E03016B
:105A70006F210201636F0201616B6BC3E9FF6CC3AD
:105A8000EAFF6BC35FF26CC360F2A4EC1AF0140E71
:105A90000201536F546B0201280E516F090E526FB1
:105AA00096EC18F0F36AF46A120027D8020E35D883
:105AB000020E38D8020E2BD8020E39D8040E2DD87B
:105AC000040E30D8040E23D8040E31D8060E25D883
:105AD000060E28D8060E1BD8060E29D80A0E1DD889
:105AE0000A0E20D80A0E13D80A0E03D83CC9EFFFBD
:105AF000120022D8010E9CEF2DF070C3E9FF71C394
:105B0000EAFF12000201E06FE16B0201120014D8FB
:105B1000E552E750EF6E7DEF2DF00ED8EFCF3CF958
:105B20007DEF2DF0E6DFEF50E66E7DEF2DF0E1DF4B
:105B30003CC9EFFF7DEF2DF0E926000EEA221200AE
:105B4000485454502F312E3020353033200D0A0D5B
:105B50000A5365727669636520556E617661696C7A
:105B600061626C650D0A000D0A0D0A00485454501C
:105B70002F312E3020323030204F4B0D0A436F6EC4
:105B800074656E742D747970653A200048545450D1
:105B90002F312E3020343034204E6F7420666F75D4
:105BA0006E640D0A0D0A4E6F7420666F756E642E5A
:105BB0000D0A00617564696F2F782D776176650035
:105BC0006170706C69636174696F6E2F6A61766170
:105BD0002D6172636869766500696D6167652F6A1A
:105BE00070656700696D6167652F67696600746538
:105BF00078742F6A6176617363726970740074657A
:105C000078742F637373006170706C696361746979
:105C10006F6E2F6A6176612D766D00746578742FD2
:105C200068746D6C00746578742F706C61696E00B7
:105C300047756573740059657300537570657220FC
:105C400055736572000D0A4E6F772072756E6E691E
:105C50006E67206170706C69636174696F6E2E2E5F
:105C60002E000D0A526561647920746F20646F778D
:105C70006E6C6F61642046696C652053797374653E
:105C80006D20496D616765202D2055736520586D25
:105C90006F64656D2070726F746F636F6C2E0D0A88
:105CA000000D0A44484350202620495020476C6587
:105CB000616E696E672064697361626C65642E0D44
:105CC0000A000D0A44484350202620495020476CC2
:105CD00065616E696E6720656E61626C65642E0D2C
:105CE0000A000D0A44656661756C74205375626E16
:105CF0006574204D61736B2028000D0A4465666150
:105D0000756C7420476174657761792041646472B1
:105D10006573732028000D0A44656661756C7420F4
:105D2000495020416464726573732028000D0A5342
:105D3000657269616C204E756D6265722028003253
:105D40003030206F6B0D0A00323236205472616E93
:105D50007366657220436F6D706C6574650D0A0023
:105D600031323520446F6E652E0D0A0031353020FA
:105D70005472616E7366657272696E6720646174D5
:105D8000612E2E2E0D0A00353330204C6F67696E60
:105D90002072657175697265640D0A0035303220B4
:105DA0004E6F7420696D706C656D656E7465640D01
:105DB0000A00353030200D0A003232312042796538
:105DC0000D0A00323330204C6F6767656420696EBE
:105DD0000D0A003333312050617373776F72642082
:105DE00072657175697265640D0A00323230205235
:105DF000656164790D0A0041424F5200504F525480
:105E00000053544F520051554954005041535300D0
:055E100055534552004E
:0A5E16001C0E0201576F586B0201C9
:105E2000000E556F090E566F52EC19F0ACEC19F0DC
:105E30000301000E836F090E846FF5D80901010E6E
:105E4000001912E1015110E10451106E116A060EA1
:105E500010180AE1115008E10551126E136A040E80
:105E6000121801E1135001E0000C020E061905E1C1
:105E7000075103E106D9EF6A0DD0010E061906E1BC
:105E8000075104E1010EFDD8EF6E04D0020EF9D8DF
:105E9000EF6E000C0201B8510901185D2EE10201FC
:105EA000B9510901195D29E10201BA5109011A5DCF
:105EB00024E10201BB5109011B5D1FE17CC3E9FF25
:105EC0007DC3EAFF08C9EEFF09C9EEFF0AC9EEFF6C
:105ED0000BC9EEFF0CC9EEFF0DC9EEFF7CC3E9FF55
:105EE0007DC3EAFF060ED7D80EC9EEFF0FC9EEFF3D
:105EF00010C9EEFF11C9EEFF010C000C010E0901E3
:105F0000006F016B026B080E036F060E046F040E28
:105F1000056F030182050BE1010E0901066F076B96
:105F200012691369146915691669176914D0020E8C
:105F30000901066F076B80C3E9FF81C3EAFFEECF5B
:105F400012F9EECF13F9EECF14F9EECF15F9EECF2B
:105F500016F9EFCF17F9BCC208F9BDC209F9BEC2E4
:105F60000AF9BFC20BF9C0C20CF9C1C20DF9B8C21F
:105F70000EF9B9C20FF9BAC210F9BBC211F97AD839
:105F8000EF500E190201C2151BE174D8010E83D81F
:105F9000EF5009010F190201C31512E16BD8020E6F
:105FA0007AD8EF50090110190201C41509E162D82D
:105FB000030E71D8EF50090111190201C51509E04E
:105FC000C6C218F9C7C219F9C8C21AF9C9C21BF961
:105FD00009D050D8EECF18F9EECF19F9EECF1AF953
:105FE000EFCF1BF90301000E836F090E846F1BD8DE
:105FF0001C0E0201626F636B0201060E616F0201EB
:10600000120E5F6F090E606FA4EC1AF01C0E0201F5
:10601000536F546B0201000E516F090E526F96ECD4
:1060200018F0FBEF1AF032D819D8F3CFEEFF11C0F9
:10603000EDFF2CD8020E2FD811D8020EF3CFEBFFB4
:10604000030E11C0EBFF22D8060E25D807D8060E86
:10605000F3CFEBFF070E11C0EBFF1200EECFD8F22B
:10606000EDCFD9F27EEC2AF0F3CF10F0F4CF11F09F
:1060700046EF30F080C3E9FF81C3EAFF060E4BEF25
:1060800030F07EC3E9FF7FC3EAFF120083C3E9FF5C
:0E60900084C3EAFF1200E926000EEA22120085
:02609E000B01F4
:1060A000BD6BBE81A3EC17F0FEEC37F0DFEC1BF00C
:1060B0003AEF04F00901010EB66F0901B65101E192
:1060C000FDD0B66B0B01BD51040A01E1D7D0070A20
:1060D00001E1A1D0050A01E187D0010A72E0050AB9
:1060E0003FE0070A36E0050A02E0010AE6E10201A4
:1060F000B50E5D6F090E5E6F0201BF0E5B6F0B0E7A
:106100005C6FF1EC19F0000915E10201160ED66F73
:1061100096EC36F0010BD1E0E3EC19F00009CDE18B
:106120000201B86BB96BBA6BBB6B0B01BE813EEC65
:106130001FF0C3D70901010EB66FB55103E10B0182
:10614000020E39D0060EB55D01E095D00B01050EAB
:1061500032D00901B66B0BEC38F00009AEE0ABD0E1
:106160000301C90E696F0B0E6A6F0301B50E676FED
:10617000090E686F0301BF0E656F0B0E666F03019A
:10618000B10E636F090E646F34EC2CF0000916E059
:106190000901010EB66FB50503E10B01030E0BD02B
:1061A000060EB55D03E10B01060E05D0110EB55DBF
:1061B00004E10B01070EBD6F80D7B66BACEC19F094
:1061C0007AD0C9CB41F1CACB42F10101B10E3F6F88
:1061D000090E406F0101BF0E3D6F0B0E3E6F6FEC5D
:1061E0001DF0000915E012D0C9CB6EF1CACB6FF1DA
:1061F0000101B10E6C6F090E6D6F0101BF0E6A6F68
:106200000B0E6B6F2DEC08F0000902E00B01BD6B6B
:106210000901B66B52D7BD6B290ED880C955000E47
:10622000CA5529E30301ED0E366F0B0E376F0301DC
:10623000EB0E346F0B0E356F0301C90E326F0B0E70
:10624000336F0301CB0E306F0B0E316F0301B50EB0
:106250002E6F090E2F6F78EC32F000090AE0080E5D
:106260000901B55D06E1010EB66F0B01040EBD6FAD
:1062700002D00B01BD6BACEC19F01FD766EC18F027
:10628000000901E11AD7EDCB40F3EECB41F3EBCBA4
:106290003EF3ECCB3FF3C9CB3DF30301CB0E3B6F99
:1062A0000B0E3C6F03013A6B0301BF0E386F0B0EF0
:1062B000396FF2EC32F00B01BD6BFFD651EC07F0F9
:1062C0004CEC1FF0030192A102D00B01BE9150EFE4
:0262D00018F0C4
:0E62D200FF0EE3CFEAFFE552FF0EE3CFE9FF38
:1062E000E552E66AE66AD9CFE6FFDACFE6FFFC0EB2
:1062F000E124D96EFF0EE220DA6EE66AE66AE66A0B
:10630000200EEF5C06E0090EEF5C03E0EF6603D0C1
:106310003FD0EE50F5D72D0EEF5C03E1FF0EE32AE0
:1063200003D02B0EEF5C01E1EE502F0EEF6424D072
:106330003A0EEF6021D0D890F90EE336FA0EE3362C
:10634000FD0EDECFE3FFFE0EDDCFE3FFD890F90EAA
:10635000E336FA0EE336D890F90EE336FA0EE3365A
:10636000FD0EE350DE26FE0EE350DD22300EEE5C25
:10637000DE26000EDD22D9D7FF0EE3CFE8FFE8527C
:1063800007E0F90EE31EE32AFA0ED8B4E306E31E93
:10639000E552E552E552FF0EE3CFDAFFE552FF0E7C
:1063A000E3CFD9FFE552E1CFE9FFE2CFEAFFED52BB
:1063B000ED52EECFF3FFEFCFF4FF1200D9CFE6FF9F
:1063C000DACFE6FFFA0EE3CFD9FFFB0EE3CFDAFF19
:1063D000FD0EE35209E72D0EDE6EFC0EE31EE32AEE
:1063E000FD0ED8B4E306E31EE652E652E652FD0E79
:1063F000E124E76EFF0EE220E46EE652F70EE3CFF3
:10640000E6FFF70EE3CFE6FF4EEC32F0F90EE124A3
:10641000E96EFF0EE220EA6E3EEC32F00AE13BEC60
:1064200032F009E13EEC32F008E13BEC32F007E1FA
:1064300008D049EC32F044EC32F049EC32F044EC54
:1064400032F049EC32F0DE6AF90EE126FF0EE2226C
:10645000FF0EE3CFDAFFE552FF0EE3CFD9FFE5529F
:10646000FC0EE124E96EFF0EE220EA6EEECFF3FFB0
:10647000EFCFF4FF1200EF380F0B1200EF500F0BAD
:1064800002E1EE52D8841200EF380F0B300FDE6EAF
:106490001200EE500F0B300FDE6E1200FC0EE3CF39
:1064A000E9FFFD0EE3CFEAFF100EE66EEE6AEE6A3C
:1064B000EF6AD890FD0EE336FE0EE336ED36ED368C
:1064C000EF36FF0EE30609E06FEC32F0EE526FECB0
:1064D00032F0EE526FEC32F0EDD7E56E1200030EA3
:1064E000EF24E8B6EF6E300EEF24E8BEEF6E000C3E
:1064F000080E0201576F586B0201000E556F090E0E
:10650000566F52EC19F002C92EF903C92FF909018F
:10651000026B036B080E0201E06FE16B0201000EDB
:10652000DE6F090EDF6FB2EC2AF0F3CF28F9F4CF5B
:1065300029F90901281F291F080E106ED9D8E85023
:10654000EF5ED6D8EF500201576F586B30C355F24B
:1065500031C356F252EC19F0CBD8EF500201E06F84
:10656000E16B30C3DEF231C3DFF2B2EC2AF0F3CFDD
:106570002AF9F4CF2BF909012A1F2B1F040E02015F
:10658000E06FE16B0201280EDE6F090EDF6FB2ECE7
:106590002AF0F3CF2CF9F4CF2DF90301000E426F4E
:1065A000090E436F7AD82EC3E9FF2FC3EAFF00C953
:1065B000EFFF34C3E9FF35C3EAFF04C9EEFF05C9A5
:1065C000EDFF36C3E9FF37C3EAFF06C9EEFF07C98F
:1065D000EDFF09012E512C1902E12F512D1901E077
:1065E000000C010C0901016B3AC300F9026B036B4B
:1065F0003EC304F93FC305F940C306F941C307F997
:1066000003013D51E66EE66A3BC3E6FF3CC3E6FF8D
:10661000080EE66E090EE66EAAEC35F0106E060E58
:10662000E15E10500301000E426F090E436F35D832
:10663000080E03013D250201E06FE16B000EE1232E
:106640000201000EDE6F090EDF6FB2EC2AF0F3CF0D
:1066500002F9F4CF03F9080E03013D2503016E6F23
:106660006F6B000E6F230301010E6D6F38C36BF368
:1066700039C36CF3E9EC2CF0080E03013D2502014F
:10668000536F546B000E54230201000E516F090E1C
:10669000526F96EC18F0FBEF1AF02FD8040E15D8B5
:1066A000040EF3CFEBFF050E1FD8060E0ED8060E14
:1066B000F3CFEBFF070E18D8020E07D8020EF3CF68
:1066C000EBFF030E11C0EBFF1200E926000EEA22D9
:1066D000EECFD8F2EDCFD9F27EEC2AF0F3CF10F066
:1066E000F4CF11F07DEF33F011C0EBFF7DEF33F00D
:1066F00032C3E9FF33C3EAFF120042C3E9FF43C3D9
:04670000EAFF12009A
:0C6704004D6F6474726F6E69782054430E
:10671000502F495020537461636B2056332E303311
:10672000000D0A507265737320616E79206B657974
:1067300020666F7220436F6E666967757261746957
:106740006F6E206D656E752E00444843502F476C68
:1067500065616E696E672E2E2E000D0A0D0A0D4DB5
:1067600078576562537276722044656D6F20417070
:10677000706C69636174696F6E2076312E302028E9
:106780004D6F6474726F6E6978205443502F495076
:1067900020537461636B2056332E30332C204175A7
:1067A000672030322032303036290D0A0D0A093187
:1067B0003A204368616E676520426F61726420739E
:1067C000657269616C206E756D6265722E0D0A09C5
:1067D000323A204368616E67652064656661756C56
:1067E0007420495020616464726573732E0D0A0928
:1067F000333A204368616E67652064656661756C35
:10680000742067617465776179206164647265736F
:10681000732E0D0A09343A204368616E676520645F
:10682000656661756C74207375626E6574206D6148
:10683000736B2E0D0A09353A20456E61626C652036
:1068400044484350202620495020476C65616E69BA
:106850006E672E0D0A09363A2044697361626C65D1
:106860002044484350202620495020476C65616EE3
:10687000696E672E0D0A09373A20446F776E6C6F88
:1068800061642046696C652053797374656D204995
:106890006D6167652E0D0A09383A205361766520CF
:1068A0002620517569742E0D0A0D0A456E746572A5
:1068B0002061206D656E752063686F6963652028AF
:1068C000312D38293A20000D0A496E76616C6964D1
:1068D00020696E70757420726563656976656420E1
:1068E0002D20496E7075742069676E6F7265642E15
:1068F0000D0A507265737320616E79206B65792083
:10690000746F20636F6E74696E75652E2E2E0D0A7E
:06691000001B5B324A008F
:0A69160054C38EF303018D6B0301DF
:10692000080E8C6F6CEF39F056C3B1F957C3B2F94A
:10693000C750040B01E0010EE5D8FAE1C580C5B0EF
:10694000FED7A1B6010C55C38FF3E1D801E0010CCD
:10695000C750040B01E0010ED5D8FAE1C5BC19D02F
:10696000B2C98FF3D4D801E0010CC750040B01E089
:10697000010EC8D8FAE1B1C98FF3C9D801E0010C02
:10698000C750040B01E0010EBDD8FAE1C5AC000C04
:10699000020C020C59C356F35AC357F358C355F3AC
:1069A000C3DF0901086FE85005E178D80901086FD5
:1069B000E85002E008511200C750040B01E0010E3C
:1069C000A1D8FAE1C580C5B0FED7A1B6010C03017C
:1069D000582903018F6F9BD801E0010CC750040BAD
:1069E00001E0010E8FD8FAE1C5AC000C020CC750D3
:1069F000040B01E0010E86D8FAE15BC38FF387D860
:106A000001E0010CC750040B01E0010E7BD8FAE154
:106A1000C5AC000C020CC750040B01E0010E72D88B
:106A2000FAE1C584C5B4FED7000C7BEC39F0C5B6DD
:106A3000FED7C59AC588C5B8FED7C95012007BECF1
:106A400039F0C5B6FED7C58AC588C5B8FED7C58496
:106A5000C5B4FED7000C5DC359F35EC35AF35CC3E3
:106A600058F398DF0901006FE85016E10301615106
:106A7000610700090EE0D9DFE66E03015FC3E9FF9D
:106A800060C3EAFF5F2B000E6023E552E750EF6E14
:106A9000EDD7D5DF0901006F00511200C750040B7C
:106AA00001E0010E2FD8FAE1C584C5B4FED7A1B626
:106AB000010C000CC750040B01E0010E23D8FAE1D1
:106AC000C580C5B0FED7A1B6010C62C38FF31FD835
:106AD00001E0010CC750040B01E0010E13D8FAE1EC
:106AE000A1B6010CC5BC03D00901B56B03D00901E7
:106AF000040EB56FC584C5B4FED7A1B6010C09015B
:106B0000B5511200106E1F0EC5141010120080EC4B
:066B100039F0000912003B
:0A6B1600FB0EE3CFF6FFFC0EE3CF09
:106B2000F7FFFD0EE3CFF8FFFE0EE3CFE9FFFF0E08
:106B3000E3CFEAFFF90EE35003E1FA0EE35009E078
:106B4000F90EE30602E2FA0EE3060900F550EE5CE8
:106B5000F1E01200D9CFE6FFDACFE6FFFA0EE3CF7D
:106B6000D9FFFB0EE3CFDAFFFC0EE3CFE9FFFD0E0A
:106B7000E3CFEAFFE9CFF3FFEACFF4FFF80EE350EB
:106B800003E1F90EE35008E0F80EE30602E2F90E25
:106B9000E306DECFEEFFF2D7FF0EE3CFDAFFE552DA
:106BA000FF0EE3CFD9FFE5521200FB0EE3CFF6FF55
:106BB000FC0EE3CFF7FFFD0EE3CFF8FFFE0EE3CFB1
:106BC000E9FFFF0EE3CFEAFFE9CFF3FFEACFF4FFDF
:106BD000F90EE35003E1FA0EE35009E0F90EE30683
:106BE00002E2FA0EE3060900F5CFEEFFF1D712003C
:106BF000FB0EE3CFF6FFFC0EE3CFF7FFFD0EE3CF76
:106C0000F8FFFE0EE3CFE9FFFF0EE3CFEAFF090036
:106C1000F550EF5C02E1EE66FAD71200FB0EE3CF0F
:106C2000F6FFFC0EE3CFF7FFFD0EE3CFF8FFFE0EFD
:106C3000E3CFE9FFFF0EE3CFEAFFE9CFF3FFEACFAF
:106C4000F4FF0900F5CFEFFFEE66FBD71200FE0E52
:106C5000E3CFE9FFFF0EE3CFEAFFF36AF46AEE52F7
:106C600003E0F34AF42AFBD71200D9CFE6FFDACFCC
:106C7000E6FFFA0EE3CFD9FFFB0EE3CFDAFFFC0EFF
:106C8000E3CFE9FFFD0EE3CFEAFFE9CFF3FFEACF61
:106C9000F4FFF80EE35003E1F90EE3500BE0F80EB9
:106CA000E30602E2F90EE306DECFEFFFEE66F1D770
:106CB000DD52EFD7FF0EE3CFDAFFE552FF0EE3CF51
:106CC000D9FFE5521200FE0EE3CFE9FFFF0EE3CF3E
:106CD000EAFFE9CFF3FFEACFF4FF610EEF5C05E6D0
:106CE0007B0EEF5C02E7DF0EEF16EE52F6E11200CC
:106CF000AA6AA96A3F0EA6160901B80E006F020E15
:106D0000016FA950106E116A120E105C000E11581E
:106D10000CE2A68000C9E9FF01C9EAFF002B000EC2
:106D20000123A8CFEFFFA92AECD71200D6C2A9FFF2
:106D3000AA6AA6B2FED73F0EA616A680A8501200D9
:106D4000D7C2A9FFAA6AA6B2FED72F0EA616A6849E
:106D5000550EA76EAA0EA76EA6820000A6B2FED799
:106D6000A69400D012001200240EAC6E900EAB6EF2
:106D7000080E7E6E02011F0E7CD8080A36E00F0A4C
:106D800032E0010A2AE0030A23E0010A1CE0070AB4
:106D900015E0010A0EE0030A07E0010A28E10901F3
:106DA000340E1C6F820E1DD009018C0E1C6F200E3C
:106DB00018D00901450E1C6F100E13D00901220EC8
:106DC0001C6F080E0ED00901100E1C6F040E09D0A6
:106DD0000901080E1C6F020E04D00901030E1C6F7E
:106DE000010E1D6F08D0AC0E03D0560E01D0AC0EB4
:106DF00009011C6F1D6B1CC9AFFF1DC910F0116A82
:106E000010507F6E12000201230E33D8926E0201E1
:106E1000240E2FD8936E0201250E2BD8D809946E1C
:106E20000201280E26D8976E0201290E22D81009D9
:106E3000986E120002012A0E1CD8896E02012B0ED8
:106E400018D88A6E02012C0E14D88B6E02012F0EF8
:106E500010D88E6E0201300E0CD88F6E1200020117
:106E6000310E07D8C16E0201320E03D87F0BC06EFF
:086E70001200D66F96EF36F018
:086E78000001EC6BE06BE16B23
:106E8000EA6BEB6B9D9A9D9812009D8A9D9812006B
:106E90000001E16BE1C0E0F0EB6BEBC0EAF0120047
:106EA000060EAB1402E0AB98AB889EAA0ED0000190
:106EB000EB51EA6AE20FE96E000EEA22AECFEFFF75
:106EC000EB2B070EEB15EB6FF0D712000001E05132
:106ED000E15D0DE0E051EA6A600FE96E000EEA2222
:106EE000EF50AD6EE02B7F0EE015E06F12009D9825
:106EF000120012000001EC5112000001EA51EA6A8E
:106F0000E20FE96E000EEA22EFCFB1F9EA2B070E8D
:106F1000EA15EA6F0901B15112000001E129106E72
:106F2000116A7F0E1016000E11160001E051126E4C
:106F3000136A1250101802E11350111802E10400F4
:106F4000ECD7F29E9DB805D0EDC0ADFF9D88F28EC6
:106F500011D00001E151EA6A600FE96E000EEA22E9
:106F6000EDC0EFFF0001E12B7F0E0001E1150001F4
:106F7000E16FF28E12000001EE519F0805E2EE393A
:106F80000F0B0F0B570F04D0EE390F0B0F0B300FF9
:106F90000001ED6FC2DF0F0E0001EE15090804E2DB
:106FA0000F0EEE15570F03D00F0EEE15300F000128
:106FB000ED6F8DEF37F00001EFC0E9FFF0C0EAFFA1
:106FC000EF2B000EF023EFCF08F9EF5004E008C9D3
:106FD000EDF0A3DFF0D712000001F1C0F6FFF2C020
:106FE000F7FFF12B000EF2230800F5CF00F9F55062
:0C6FF00004E000C9EDF091DFEFD71200C3
:046FFC000B01EF6B2B
:10700000F069F169F269F369F469F569F66BF76B98
:10701000F86BF96B12000B01EF5129E10301260E09
:107020007E6F090E7F6F03011C0E7C6F090E7D6F52
:107030000BEC2FF000092CE00901265115E11CC9C9
:10704000F0FB1DC9F1FB1EC9F2FB1FC9F3FB20C9F0
:10705000F4FB21C9F5FB22C9F6FB23C9F7FB24C9C0
:10706000F8FB25C9F9FB010C0B01010EEF6F66EC73
:1070700018F000090CE00301826B03011C0E806F05
:10708000090E816F7EEC2FF00B01EF6B010C000CF1
:10709000010CFACBE9FFFBCBEAFFEECF22F9EECFF2
:1070A00023F9EECF24F9EFCF25F90301010E826F0A
:1070B00003011C0E806F090E816F7EEF2FF0FCCB59
:1070C000E9FFFDCBEAFF0B01F651EE1808E1F7519D
:1070D000EE1805E1F851EE1802E1F951EE1814E04E
:1070E0000201C6510B01F65D20E10201C7510B01FF
:1070F000F75D1BE10201C8510B01F85D16E10201C9
:10710000C9510B01F95D11E1FECBE9FFFFCBEAFFAD
:10711000F0CBEEFFF1CBEEFFF2CBEEFFF3CBEEFFC9
:0C712000F4CBEEFFF5CBEEFF010C000CF1
:04712C00545854005F
:1071300048544D00434C4100435353004A53000010
:1071400047494600434749004A5047004A415200D8
:1071500057415600545854005A5458005A48540045
:107160005A434C005A4353005A4A5300485454500F
:107170002F312E3020323030204F4B00436F6E7451
:10718000656E742D747970653A2000436F6E746576
:107190006E742D456E636F64696E673A20677A6915
:1071A000700D0A00457870697265733A20300D0AD7
:1071B0000043616368652D436F6E74726F6C3A2093
:1071C0006D61782D6167653D3330302C206D7573AE
:1071D000742D726576616C69646174650D0A00478F
:1071E000455400494E4445582E48544D004C4F4795
:0771F000494E2E4347490000
:0871F8002A0EF66E080EF76E78
:10720000000EF86E03010900F550776F0900F55084
:10721000786F03E1776701D03DD00900F550726FB8
:107220000900F550736F0900F550746F09000900EB
:10723000F550E96E0900F550EA6E090009000900F1
:10724000F550756F0900F550766F09000900F6CF0B
:1072500079F3F7CF7AF3F8CF7BF372C3F6FF73C3FA
:10726000F7FF74C3F8FF0301755302E1765307E09B
:107270000900F550EE6E7507F8E27607F9D779C385
:10728000F6FF7AC3F7FF7BC3F8FF03017707000E11
:06729000785BBFD712007D
:0A7296004E6F7420496D706C656D39
:1072A000656E7465640073656C6563746564006322
:1072B0006865636B65640064697361626C65640032
:1072C0003C212D2D002D2D3E006F6E006F66660057
:0772D0005570646174650054
:0872D8003F0EC716C66AC56A25
:1072E00003018C51C6128D51C71294869488C68AA8
:1072F0008EC3C8FF1200C586C7A0FED7C9501200B2
:0E7300008FC3C9FFC6BEFF0CC7B0FED7000C7E
:02730E00FF0E70
:10731000E3501D6EEF0E01D0F30EE76EE72E8EEFF9
:1073200039F00C0E1C6EE76AE72E94EF39F01C2E34
:0C73300093EF39F01D2E8CEF39F01200A5
:04733C00036A026A74
:10734000100EE76ED89006360736023603360B501D
:10735000025C0C50035805E30B50025E0C50035ABC
:08736000062AE72EF0D7120007
:087368000301856B866B876B46
:10737000886B896B8A6B580ED66E9E0ED76E010E87
:0A738000D56ED58EF284F28A120059
:06738A00036A080EE76E25
:10739000D890073603360C50035C02E3036E072ACD
:0673A000E72EF7D71200F2
:0A73A6001CEE00F02CEE00F0F86A77
:0E73B0000F9CFCEC38F0D9EC27F0FDD7120052
:0273BE00FF0EC0
:1073C000E350E84E1200000000D000D000D0E82EBC
:0473D000FAD71200D6
:0673D40056322E34330096
:0673DA0056332E30340092
:1073E0002D5D165DFA5CE25CC25CA15C625C455C92
:1073F0000000000000000000000000010003000584
:07740000000200040000007F
:02740700000083
:07740900255C1B5C075CFE23
:107410005BEE5BE45B1B5CD95BC05BB35B255C250F
:107420005C1B5C075CFE5BEE5B8C5B6C5B675B40D4
:017430005B00
:0F743100105E0B5E065E015EFC5DF75DEB5DD3EA
:107440005DC35DB95DB25D9C5D875D6C5D605D48EF
:037450005D3F5D40
:0474530000FF000036
:020000040030CA
:0100010026D8
:0100020006F7
:010003000AF2
:010005008179
:010006008178
:010008000FE8
:010009008076
:01000A000FE6
:01000B008074
:01000C000FE4
:01000D0000F2
:0200000400F00A
:10000000C0A801960004A3000000FF000000C0A8E3
:1000100001960401280300C0A80196C0A801960714
:10002000000700FFFFFFFFFFFFFF000000000000D0
:1000300000032E000061646D696E0000000070779F
:0700400000000000000000B9
:00000001FF
